:020000040800F2
:10500000F81B0020D550000869890008B980000805
:105010000000000000000000000000000000000090
:10502000000000000000000000000000BD97000824
:10503000000000000000000031910008F99800080D
:10504000E7500008E7500008E7500008E750000864
:10505000E7500008895D0008E7500008E7500008A5
:1050600000000000E7500008B15C0008E7500008AD
:10507000E7500008D985000800000000E75000084C
:1050800000000000E75000080000000000000000E1
:10509000E750000800000000E7500008E750000853
:1050A000E7500008E7500008E7500008FDA100089D
:1050B000E7500008E7500008000000000000000072
:1050C0000348854600F040FD0048004771B50008E0
:1050D000F81B00200448804704480047FEE7FEE72D
:1050E000FEE7FEE7FEE7FEE795990008C1500008DD
:1050F00030B50B46014600202022012409E00D4670
:10510000D5409D4205D31D469540491B25469540F7
:1051100040191546521E002DF1DC30BDF0B51FB40C
:105120000646002082B005464024019100901BE015
:10513000019922460F46304600F0F0FB049A059B89
:10514000801A994110D310461946224600F0D6FB2A
:10515000361A8F410197224601200021009F00F05E
:10516000CDFB38184D4100902046641E0028DFDC3E
:10517000019B00982946324607B0F0BD03460B4319
:105180009B0703D009E008C9121F08C0042AFAD2FD
:1051900003E00B780370401C491C521EF9D2704783
:1051A000D2B201E00270401C491EFBD270470022BF
:1051B000F6E710B513460A4604461946FFF7F0FF16
:1051C000204610BD30B504460020034600E05B1CBD
:1051D000934203D2E05CCD5C401BF8D030BDF8B503
:1051E00002464A40D40F42004B0052085B089A42E4
:1051F00002D20246084611464A0023D0C30D4A0097
:10520000DDB2120EAD1A202D35DA49020126490A07
:10521000F6058A19002C00D0524220214F1B11465E
:10522000B9402A411018C20D9A4221D0002C17D043
:10523000012D08DCDA05801AD20F8019D207DBB203
:1052400000F098FBF8BDDA05801A012340001B0628
:10525000C01880185A428018CA0F1043490007E04E
:105260004908C2071143DA05801A801940088018DE
:1052700000F078FBF8BD61000122511A001BF7E72E
:105280000122D2075140AAE70122D2075040A6E7E7
:10529000024670B54A40D30FDB0740002DD04A00CC
:1052A0002AD0010E140E000212020919400A520AF5
:1052B0008418E50104465443000A120A2E045043A0
:1052C000A4194219200CC543AA18120C0125AD03DC
:1052D000521C521912047F39240400D0521C10436E
:1052E00001D44000491EC2B20C06C0092018401C5F
:1052F0004008802A02D003E0002070BD4008400032
:10530000002900DA0020184370BD70B502464A40FB
:10531000D50F40004A00ED0740085208002814D07D
:10532000002A12D0C40DD30D41020120C005520243
:10533000490A520AE41A091812187D34914201D31D
:10534000641C00E04900002C01DA002070BD00233D
:10535000914201D3891A0343400849000028F7D13C
:1053600000290AD0914202D10121C90705E09142EA
:1053700001D2012101E00121C943E005C018401913
:1053800000F0F0FA70BD420005D04200120E524209
:105390008A4201DB00207047C905081870470000E9
:1053A000F0B507460846584087B0C00F0490480043
:1053B0000E46590040084908BC1A884105D23846B3
:1053C00031461E4617460B46024658004008104319
:1053D0004CD0300D039040055900400D490D05900B
:1053E000401A0290402872DA18030121000B0905C7
:1053F0000843019004980092002805D00199524278
:105400000020884100920190029840210A1A0199D7
:10541000009800F073FA05460C466B4607CB00F087
:105420008EFAC0197141039A0E0D0023D71756400A
:105430001A467A40164344D0049A002A2DD0029A84
:10544000012A039A15DC1205C01A9141012636057E
:10545000001C7141D20F059ED20700930192029663
:105460002A46234600F0CCFA07B0F0BD3846314654
:10547000FAE71605224A0F46B218C01AB7410121B1
:105480000905001C4F4100187F4111461818794149
:10549000E20F10436D19644113E0E2076D081543F4
:1054A0006408C2071443039A01261205C01A9141E9
:1054B0003605001C7141CE07400830434908C0182A
:1054C00051412A46234600F08EFACDE7FFE70498C3
:1054D00001224000C117121A00238B410498314663
:1054E000C417381AA141EEE730B40124E407634041
:1054F00030BC55E730B40124E407614030BC4FE7CD
:105500000000E0FFF0B51FB488B00B9909980024A3
:1055100048400999C00F490049080991C0070B99F3
:105520000090490049080B9109990898A64608433C
:105530001CD00B990A98084318D009980124400000
:10554000420D4800410D099824050003000B20433B
:1055500009900B980003000B20430B9050181C4936
:105560004018002201901446104605E00020014634
:105570000DB0F0BD032801DA034600E003239C468A
:10558000C11A0AAE0AE05F0008ADED5B4F00F75BA1
:105590007D430027AA187C41491C5B1E6145F2DD52
:1055A000410004AB5A522104120C0A43240C401C43
:1055B0000828DFDB01980290009970460191009065
:1055C000059B049A0799069800F01AFAD0E70000A4
:1055D0000DFCFFFFF0B50C465C4085B0E40FE4071E
:1055E00003944C000026640859009446490802467A
:1055F0000296224321D062460A431ED06200570D14
:105600004A000E032303550D012402462C492405AC
:10561000781B1B0B360B4018234326436146009032
:105620001C46501AB44103D30098401C009002E07D
:10563000921800985B41002803DA0020014605B06B
:10564000F0BD0020012109050746864611E06446A9
:105650001D46141BB54106D36546521BB341744623
:1056600007430C43A646CD07400849082843921833
:105670005B4105460D43EAD11046184313D06046FE
:10568000194650407140084306D06046101AB34195
:1056900006D20122002306E000220123DB0702E0FC
:1056A0000122D2435310009874460105381C614111
:1056B000029C039D0019694100F095F9BFE70000C5
:1056C000FD03000070B54B005B0803430BD04B009B
:1056D0005C0D002633466542B341D417AD1AA34191
:1056E00002DB0020014670BD12053018514170BD2B
:1056F000C217C10F504010B54018CA0796230021A9
:1057000000F038F910BD10B500229623114600F0C4
:1057100031F910BD0EB5C217C10F5040CA0740186D
:105720000021054B0293019200910A460B4600F0BE
:1057300067F903B000BD0000330400000EB5054951
:105740000291002100910A460B46019100F058F9A0
:1057500003B000BD33040000C20F4100400201232A
:10576000400ADB05D207090EC0187F2901DA0020A4
:105770007047962903DC9623591AC84001E09639F0
:105780008840002AF4D04042704741004002012284
:10579000400AD205090E80187F2901DA00207047DF
:1057A000962903DC9622511AC840704796398840E2
:1057B0007047000070B5CD0F4A0009030123090BA3
:1057C0001B0519430B4BED070024520D9A4201DAD9
:1057D000002070BD074B34339A4203DC9A1A00F064
:1057E0009DF802E00449511888402C43F1D0404212
:1057F00070BD0000FF030000CDFBFFFF4A0009035E
:105800000123090B1B051943094B10B5520D9A4290
:1058100001DA002010BD064B34339A4203DC9A1A99
:1058200000F07CF810BD03495118884010BD0000FD
:10583000FF030000CDFBFFFFC20FD207400040086E
:105840000BD0C10D0723DB01C91840020905400A2E
:105850001143C208400711437047002001467047BA
:1058600010B5002904DB0124E40740428C412146A5
:10587000002B04DB1C460123DB075242A3418B4271
:1058800000D1824210BD000010B5002904DB0124C4
:10589000E40740428C412146002B04DB1C460123D7
:1058A000DB075242A341994200D1904210BD000053
:1058B000CB0FDB07490010B5490802460A4307D061
:1058C0000A0D07240903E401090B121B002A01DC5D
:1058D000002010BDC900440F0C43C100E018D205E0
:1058E000801800F03FF810BD0122D207002800DB2D
:1058F000101A002900DB511A8142704710B5202A86
:1059000004DB0146203A9140002010BD9140202345
:105910009C1A0346E3401943904010BD10B5202A5D
:1059200004DB0846203AD040002110BD0B46D3408E
:10593000D0402024A21A91400843194610BD10B54A
:10594000202A06DBCB170846203A1041C1170B432B
:1059500006E00B461341D0402024A21A9140084390
:10596000194610BD002904DA401C490001D1400845
:105970004000704770B40024050C05D110240004C9
:1059800002D1002921D01124050E01D100020834D2
:10599000050F01D10001241D850F01D18000A41C39
:1059A000002801DB4000641C002908D020252E1BA4
:1059B0000D46F540A14000D00121294308430106CE
:1059C0001B1B000ADB1D02D5002070BC7047DB05E5
:1059D000181880180029F8DA401C4900F5D170BC6D
:1059E00040084000704710B5002B08DA0024401C26
:1059F000614192185B411A4301D14008400010BD3B
:105A0000F0B51FB482B005460C0003D0084604F080
:105A1000A9FC02E004F0A6FC2030024600902146DA
:105A20002846FFF76BFF049B059A04460F46184370
:105A30001143084314D0184610431BD0009840214E
:105A40000A1A18460599FFF769FF05460E46009A9F
:105A500005990498FFF752FF084305D0012004E0A0
:105A60002046394607B0F0BD0020C11705430E435C
:105A70002C43374300990E986305401A7905E40AD0
:105A800000220C43FD0A0A3002D500200146E9E756
:105A90000105101969410C9C0D9D00196941FFF722
:105AA000A2FFDFE7FEB500231A461B1A8A4103DB7B
:105AB0000020014603B0F0BD4A000D0301212D0B6B
:105AC0000905520D0D43D10702D100186D41521E38
:105AD0005110FF31FF310131002704463E46384660
:105AE000009701910246012100200905FFF716FFEA
:105AF000C3197141F818324684468E464A416146C0
:105B00002846611A904104D36046241A954176468E
:105B10001F46241900986D41401C00903428E1DD97
:105B2000F91930467041091BA84103D20022D24323
:105B3000134601E00022134601980105381C71410B
:105B4000FFF751FFB6E70000064C0125064E05E0C1
:105B5000E36807CC2B430C3C98471034B442F7D38E
:105B6000FFF7B2FA58C4000878C4000870B58C1862
:105B70000578401C6B075B0F01D10378401C2A118C
:105B800006D10278401C03E006780E70401C491CC8
:105B90005B1EF9D12B0705D40023521E0DD40B70C8
:105BA000491CFAE70378401CCB1A921C03E01D78CD
:105BB0000D70491C5B1C521EF9D5A142D8D30020A0
:105BC00070BD000038B50446064805490068FFF777
:105BD0008FFA604300E0401E00900028FBD138BDE2
:105BE00040420F0084010020F8B504460068816837
:105BF0008907890F012902D10168C90722D181686B
:105C0000114A10261140012500290ED1816829432F
:105C100081600120FFF7D6FF01F028F807460CE06D
:105C200001F024F8C01B0A2807D9606D3043606575
:105C3000A06D2843A0650120F8BD20680068C0431E
:105C4000C007EDD10020F8BD170000801FB50B483C
:105C500000900B4801900B4802900B480390694656
:105C60000A4804F075FF0A4A08481146083904F04A
:105C70005DFE00F06FFA002004B010BD61C20008A4
:105C80003DC200089DC200089BC200089001002090
:105C90001000002010B500231A4603E0845CE318CE
:105CA0009BB2521C8A42F9D3D84380B210BD000087
:105CB00010B5034800F096FD024800F093FD10BDBA
:105CC000981700205017002030B5446C1C252C403C
:105CD0000125A540046C6560046863608368102B2F
:105CE000036803D099600068C26030BD9A600068A4
:105CF000C16030BD1449012048720A4602205E325C
:105D0000507203203C3A507204200E3A50720F48F1
:105D10000D4B0078087022310870203108770C494B
:105D20005A1C087858714978997123331871597140
:105D3000203318775977107551751A461E32107531
:105D40005175107651767047E81100203E01002011
:105D50006001002010B503F007FD202003F0C2FD14
:105D6000012005F05FF9002003F0BCFD044804F0B9
:105D7000FDFF044805F0ACFA002005F0E1FA10BD83
:105D80000001002083800000F8B503F0B9FD052074
:105D90000121000700F056FF0025144C002800D018
:105DA0006560134E0221304600F04CFF002815D1EB
:105DB000012020700F48808F00280ED00127BF02DD
:105DC00000223946304600F04AFF0A2004F01EFD4A
:105DD00001223946304600F042FF6560012000F0A4
:105DE00069FE022000F066FEF8BD00007001002090
:105DF00000040050E80D00207047000010B508496D
:105E000000224A6107494B684C1523434B604B689D
:105E1000082423434B60C009C001026010BD00008C
:105E2000E0170020002002407FB500250C46064602
:105E3000039500F00FFEE009029003A9019600957A
:105E4000684600F09FFD002804D000F0D7FD002038
:105E500004B070BD00F0D2FD0120F9E710B50023B9
:105E600002E0C45CCC545B1C9342FAD310BD00002A
:105E700010B5214A00219069C305204804D5416925
:105E8000022319434161911593699B0505D5436927
:105E90000124234343616302194393695B0505D5DC
:105EA0004369082423434361E301194393691B05B4
:105EB00005D543690424234343616302194393696D
:105EC0009B0405D5436910242343436163021943AE
:105ED00093699B0304D5446920231C4344611943FF
:105EE0009369DB0305D54369402423434361A00242
:105EF0000143916110BD000000200240E017002026
:105F000070B5054600F0B2FE0646184C0AE0681C63
:105F100008D0002D04D000F0A9FE801BA84201D9B2
:105F2000032070BDA069C007F1D1A069800701D529
:105F30000220A061A069C00511D4A06980050ED41B
:105F4000A06940050BD4A069000508D4A0698004AD
:105F500005D4A069800302D4A069C00303D5FFF76C
:105F600087FF012070BD002070BD000000200240AE
:105F7000F8B51746002605460C4600F06BFD09E013
:105F800029460220226800F047FD002804D1241D84
:105F90002D1D361DBE42F3D300F030FDBE4201D2AE
:105FA0000020F8BD0120F8BD10B5084902460020C8
:105FB000054B497905E044001C5B944203D0401C2A
:105FC000C0B28842F7D310BD8C13002070000020AF
:105FD00010B500F03CFE10BD10B5094801F05CF8AA
:105FE00080B2FFF7ABFB074A074BFFF78BFA0022A3
:105FF000064BFFF7EFFAFFF701FC80B210BD00007F
:1060000004160020F853E3A59B843E4000408F40D7
:1060100070B50024204603F023F847494748A20002
:10602000641CE4B28150142CF9D3464944480A79DF
:1060300002754979417544490A7802764978417672
:106040003F490520133148720A2005F031F97D20BF
:10605000400105F047F93A49002213310C2005F0C0
:1060600011FA00210C2005F01FFA384801F014F84D
:10607000344C0125223C2085AD0309E0334801F072
:106080000BF880B22085E18EFF392D39884206DB7E
:10609000E18E80B28842F1D349198842EED80220BD
:1060A00005F056F9002002F0DBFF294D00210F20FA
:1060B00005F07EF828422064F8D0206C411C38D0CE
:1060C000400435D58122D20100210F2005F0AFF91F
:1060D0000021102005F06CF841061948490E0022F5
:1060E000C73005F09BF8164DC735687A05281FD1D3
:1060F00002221549681DFFF765F8002818D11148DC
:10610000AE7C66710422691C3630FFF737F82946E9
:106110001331084672000D466930FFF72FF8607999
:106120002946420005484838FFF728F80320207028
:1061300070BD04F08BF90000FFFF0100EC1300209C
:106140004912002092000020600100200416002067
:1061500000D0272410B5144C1448224610321146A2
:10616000083904F0E3FB0022114BE168A068FFF757
:1061700031FA104A104B05F003FB00220F4BFFF7DA
:10618000B9F900220E4BFFF7BDF9FFF791FB206034
:1061900000221346E168A068FFF762FB01D0206887
:1061A00010BD0020206010BD0000002090010020E4
:1061B00000AA8F406C45D9CC955BC83F0000F03FEA
:1061C00040A5E54010B5084800F096FA0A210648B7
:1061D00000F032FA044800F01DF9800503D50248AA
:1061E00000F01AF980B210BDA8150020F8B52F4DA7
:1061F00000220121284600F032FDFFF7E3FFFFF700
:1062000082FA2B4E3146FFF780F82A4C0122A0601B
:106210001146284600F023FD2749A0680025884242
:106220003EDB2078254F002815D02570FFF7CAFFE8
:10623000FFF769FA3146FFF768F8A060FFF7FCFA4C
:1062400000223B46FFF750F900221D4BFFF75AF999
:10625000FFF72EFB6060A068FFF7EEFA00223B46D6
:10626000FFF742F9174A184BFFF74CF906460F465D
:106270006068FFF7E1FA134A144B5242FFF742F904
:1062800032463B46FFF78CF8FFF712FB104960607F
:10629000884201DD616004E0FF21C905C84200D3E6
:1062A00065606068FFF771FAC0B2F8BD0004005085
:1062B00000401B44480000200000604000000C40EB
:1062C00000E064403333333333B33040CCCCEC3F65
:1062D0000000C842F8B5054604464035287C002633
:1062E000012808D001202874206881688907890F57
:1062F00001290ED101E00220F8BD0168C90708D0CC
:10630000606D202108436065012600202874304616
:10631000F8BD616DFF220132914302221143616594
:10632000C1688907890F0091C16889088900C16027
:106330002068816892071143816000F097FC07464E
:106340000EE000F093FCC01B0A2809D9606D022101
:106350008843102108436065002028740120F8BD9F
:10636000206880680028ECDB2068C168009A11432F
:10637000C160606D80088000401C6065C5E700005A
:10638000F8B506460D464036317C01290DD0012175
:10639000317401688A68520709D5416D2022114382
:1063A0004165002030740120F8BD0220F8BD174B74
:1063B0006A68D80547109A42154C8A6A2B6812D031
:1063C0005B035B0B1A438A622968490305D5A16800
:1063D0000143A1600A20FFF7F5FB2868800312D56E
:1063E000A06838430EE05B035B0B9A438A6229681E
:1063F000490302D5A1688143A1602868800302D5C2
:10640000A068B843A06000203074F8BD01100000FF
:1064100000270140406D70470068006C7047000025
:1064200070B5040006D0606D264600254036002871
:1064300002D006E0012070BDA5653574204600F04D
:10644000D3F8606DC00603D421688868400705D57D
:10645000606D1021084360653574EBE7606DFF22C5
:106460000132904302221043606588688207920FD0
:106470005B48012A02D10A68D2072BD10323626844
:106480009B079A4205D05B429A4202D05B009A4237
:1064900009D10A69920092080A6121680A69636851
:1064A0001A430A610CE00A69920092080A61816845
:1064B0000F22920491438160816862681143816078
:1064C0002168CA6818239A43CA602168CA68A36809
:1064D0001A43CA6081680122520691438160816833
:1064E000A28E52061143816020688168C90004D4DD
:1064F000816801221207114381602068C168394A0E
:106500001140C1602069E168022825D000200143C4
:10651000204620300278037B52035B001A4311436C
:10652000226B1143A26992031143E269D203114322
:106530002268D3681943D160616A0A46FF3AC23AB9
:1065400005D0A26A11432268D3681943D16042780A
:106550000121012A02D00BE00420D8E700780028AE
:1065600023D0606D202210436065A06D0843A065B4
:10657000E06B012820681FD00169C90703D00169B9
:1065800049084900016120684169C908C9004161A1
:1065900020684169A26B11434161A565606D800867
:1065A0008000401C6065002070BD2068C268012327
:1065B0001B041A43C260DBE70269FF239B009A4376
:1065C000026120680269236CA66C1A43636C334332
:1065D0001A430261206802690A430261D3E700009E
:1065E000002701401902FEFF10B586B004461421B1
:1065F0006846FEF7DCFD0E492068884216D10D483A
:10660000416B421511434163C16A01221143C162CA
:10661000C06A694610400590022000900320019056
:10662000002002900520000700F050FA06B010BDCF
:106630000024014000100240F8B504464069254698
:1066400040350E4608280BD02068C068C00709D026
:10665000606D202108436065002028740120F8BD8A
:10666000082700E00C2700F001FB009011E0701CEF
:106670000FD0002E05D000F0F9FA0099401AB04270
:1066800007D9606D04210843606500202874032049
:10669000F8BD206800683842E9D0606D01214902E8
:1066A000084360652068C16809058A0F0C21002A2B
:1066B0001BD12022125D002A17D10268120714D5BF
:1066C000826853070122002B08DB43688B43436039
:1066D000606D130298431043606506E0606D2023EF
:1066E00018436065A06D1043A065A069002801D122
:1066F000206801600020F8BD70B5044621680020C4
:106700008968490721D425464035297C01291CD0B8
:1067100001212974E169012904D02046FFF764FAB8
:10672000002811D1616D0A4A1140FF220132114344
:1067300061650021A165297422681C21116021680E
:106740008A6804231A438A6070BD022070BD00006D
:10675000FEF1FFFF30B5014620314A790023022ABD
:1067600004D00422C2630B71012030BD026814689A
:106770000E25AC4314600268146864086400146059
:10678000446C1C22144001221546006CA540456053
:106790004A7118460B7130BD70B500240146203196
:1067A0004A79022A03D00421C163012418E0026857
:1067B00013680E25AB431360026813685B085B0027
:1067C0001360436C1C221340012215469D40036C4C
:1067D0005D604A7100220A71816B002900D08847F0
:1067E000204670BDF0B4016C0D6801680C68466C01
:1067F0001C2304221E401746B7402F420ED06707C5
:106800000CD50C68A40602D40C6894430C60416C4F
:1068100019408A40016C4A60016B1AE00227B740B8
:1068200002462F402032002F17D0A70715D50C683D
:10683000A40605D40C680A25AC430C6001215171F3
:10684000446C02211C40036CA1405960002111716D
:10685000C16A002918D0F0BC08470827B7402F426A
:1068600012D0240710D50C680E25AC430C60446C84
:1068700001211C400B46A340046C6360C16351714D
:1068800000211171416BE4E7F0BC704770B5040062
:106890003CD01F48256814212818FEF729FC8000E9
:1068A00060641C4820640221204620300246417169
:1068B00029681948E3680140A0686669184323699C
:1068C00033431843A3691843E3691843236A184301
:1068D000084328600121A0688903884210D00D4830
:1068E0008030836A656C1C210D400F26AE40B34397
:1068F0008362656C63680D40816AAB400B438362C1
:106900000020E06301215171107170BD012070BD44
:10691000F8FFFDBF000002400F80FFFFF8B50446FE
:106920008C46203001790025012909D00126067105
:1069300041790027012905D0077102252846F8BDB5
:106940000220F8BD02214171E7632068016849080F
:106950004900016061462046FFF7B6F9206B002828
:106960002068016801D00E2205E0042291430160F5
:10697000206801680A2211430160206801683143E0
:106980000160DBE7F8B51A4E0546307C0F4601285A
:1069900007D0012030741748FFF7B2FA010002D087
:1069A00021E00220F8BD0020C04338606C6814E08C
:1069B0002046FFF723FA0F48FFF7A2FA01460E48D8
:1069C000426808239A434260426843159A434260F2
:1069D000002901D03C6006E08034A8686A68C001E4
:1069E0008018A042E4D8002030740846F8BD0000AA
:1069F000E017002050C30000002002400548416815
:106A0000022211434160416801221143416000208C
:106A10007047000000200240F8B50C4C1646207C60
:106A20000F46012808D0012020740948FFF768FAB2
:106A30000025002802D006E00220F8BD65613E6016
:106A40000348FFF75DFA2574F8BD0000E017002049
:106A500050C3000011484168C9070BD0EFF3108103
:106A600072B60F4AC2600F4AC26081F31088416853
:106A7000C9070ED1416889070DD5EFF3108172B6B1
:106A8000094A0261094A026181F31088406880075F
:106A900001D501207047002070470000002002400F
:106AA000EFCDAB8905040302BFAE9D8C1615141300
:106AB0007047000010B504494A69024202D048619B
:106AC000FFF7F6FF10BD000000040140FCB50023F5
:106AD0000124A2E027462A469F403A406FD04D68E5
:106AE000012D05D0022D03D0112D01D0122D16D16C
:106AF00085680326AC465D00AE46AE406546B543AC
:106B0000AC46CE687546AE4065462E438660466804
:106B10000D79BE43ED06ED0F9D4035434560C668D7
:106B20005F000325BD40AE46AE4335468E68BE408D
:106B30002E43C6604E68022E01D0122E14D1DE08FC
:106B4000B60036180196366A5D07B446EE0E0F257C
:106B5000B54000966646AE43B4460D69009EB5400A
:106B600066462E43019D2E6206687546AE430D793A
:106B7000AD07AD0FBD40354305604D68ED004BD509
:106B8000294D6E6B26436E639E08284DB60075191D
:106B9000AC46AD689E07360F0F27B740BD430527AB
:106BA0003F07B84201D1002715E0214FB84201D17B
:106BB000012710E01F4FB84202D102270BE02BE063
:106BC0001D4FB84201D1032705E01C4FB84201D147
:106BD000052700E00627B7402F436546AF60184DF4
:106BE0002E684F689643FF0300D516432E606E68EB
:106BF0004F689643BF0300D516436E60AE684F687A
:106C00009643FF0200D51643AE60EE684F68964388
:106C1000BF0200D51643EE605B1C0A681546DA40D9
:106C200000D057E7FCBD000000100240000001400A
:106C30000004005000080050000C0050001C0050E0
:106C4000000401400069084000D0012070474269FB
:106C500013460B401B0491430B4383617047002A8A
:106C600001D08161704781627047000001488068EF
:106C70007047000078010020024881680278891876
:106C8000816070477801002010B508480024016831
:106C9000402211430160204600F00AF8002801D08C
:106CA000012401E000F042FA204610BD002002401D
:106CB00070B504460D4D7D202978C000FEF718FA06
:106CC00001460B480068FEF713FA00F02BFF00287E
:106CD00009D1042C07D200222146401E00F04EFAB2
:106CE00000206C6070BD012070BD000078010020A4
:106CF0008401002070477047F8B502F001FE604C37
:106D00000120E070208AFEF7FEFC01467F20C005CE
:106D1000FEF7FBFA5B4D06462968FEF760FA28602D
:106D20000120A16AC005814201DA084603E030462D
:106D3000FEF7AAFAA062FF21C9050025C84200D3C8
:106D4000A562607800280BD102214F48FFF77AFF37
:106D500002004E494E4817D00022FFF780FFE5623F
:106D600002214948FFF76EFF4A4E002855D0E562E0
:106D7000B08AFEF7C8FC434F3968FEF7B5FD5FD215
:106D80004549012008705DE00122D1034048FFF72A
:106D900066FF208AFEF7B7FC01467F20C005FEF79C
:106DA000B4FAE16AFEF71BFA3C49E0628842D7DD9B
:106DB00038480127F926403000900A213046FEF776
:106DC00097F9002903D131493148FFF701F9022130
:106DD0002D48FFF737FF002801D0002701E0002FE2
:106DE00012D102212848FFF72DFF00280CD104F012
:106DF0008FFC00990120888005F0E6F9642003F0FB
:106E000005FD28492648C8600A2003F0FFFC3046EB
:106E1000761EF6B20028D0D1A2E7208AFEF773FCD6
:106E200001467F20C005FEF770FAE16AFEF7D7F948
:106E30001D49E06288429BDB1A491948C86097E700
:106E400015480570708F401EFEF752FC3968FEF73A
:106E50004BFD06D82079002803D014490120087082
:106E600001E012480570708FFEF74DFC3968FEF79F
:106E70003BFD04D22079002801D004F00DFCF8BDC0
:106E80003C0100207401002000040050008000003C
:106E900000000050E80D0020760000200000404077
:106EA0000400FA0500ED00E00000A040860000208C
:106EB000704770B5040010D0022025462035A87315
:106EC000204601F091FBA87B032805D0204600F066
:106ED000B9F80020A873687370BD012070BD7047B9
:106EE000704710B5044600680168C943C90708D156
:106EF0008168C943C90704D1012141602046FFF7D9
:106F0000FBFE20680168C943890708D48168C9432A
:106F1000890704D4022141602046FFF7EBFE206878
:106F20000168C943490708D48168C943490704D4A3
:106F300004214160204600F0F7F820680168C94349
:106F4000090708D48168C943090704D408214160AE
:106F50002046FFF7ADFF20680168C943C90608D481
:106F60008168C943C90604D4102141602046FFF757
:106F7000C2FE20680168C943890608D48168C943F4
:106F8000890604D4202141602046FFF7A9FF20682C
:106F90000168C943490608D48168C943490604D435
:106FA000402141602046FFF79AFF10BDF8B504006C
:106FB00005D025462035A87B002802D006E0012018
:106FC000F8BD00206873204600F04EF80220A87338
:106FD0002068C26884466368012B01D10620824381
:106FE00016486169814202D0072040038243002B8A
:106FF00001D1D82082431248A66802401846304387
:10700000676A266A3E433043A66A30431043002B2A
:1070100002D0012B04D005E02369E2691A4300E0A5
:10702000E2681043054A914202D0A2691143084325
:107030006146C8600120A8730020F8BDFFFF000072
:10704000F8F119FF10B500680549884207D10548D5
:10705000816B4900490881630D2000F073F810BD71
:10706000007C00400010024010B5006808498842CA
:107070000CD10848816BC2041143816300220121B5
:107080000D2000F07BF80D2000F06CF810BD000022
:10709000007C0040001002400068C069704700009A
:1070A000F8B504460220254620351746A8731D482A
:1070B0000268C3041A4302602068C2689B121A4324
:1070C000C2602068026901263243026122681020F2
:1070D0005060206881611021204601F0F5FA0328F4
:1070E0001FD0216808204860206847610821204699
:1070F00001F0EAFA032814D0204601F075FAA87BC3
:1071000003280ED0206881683143816020680169BE
:107110003143016120680169042211430161AE73AA
:107120000020F8BD00040140704700000448416B96
:10713000012211434163816B020411438163704753
:1071400000100240002809DBC106C90E012088405A
:1071500003490860BFF34F8FBFF36F8F7047000084
:1071600080E100E0002805DBC106C90E012088404F
:10717000014908607047000000E100E010B503F02D
:1071800043F910BD02494A6882434A6070470000D3
:107190000070004002480168821511430160704789
:1071A0000070004002494A6802434A60704700008C
:1071B0000070004005480168022211430160044844
:1071C000016904221143016130BF70470070004023
:1071D00000ED00E0F0B5154A1368154D54152D6A01
:1071E0002340ED07ED0F002B04D0002D02D01668D0
:1071F000A64316601668B608B600064316600D482A
:10720000076904263743076101290DD040BF20BF1D
:1072100020BF0169B1430161002B04D0002D02D0D1
:10722000106820431060F0BD30BFF2E700700040EE
:107230000000014000ED00E0F8B5044600780027AA
:10724000534D800671D5524E403EB06BC00004D401
:10725000B06BA9050843B06301274E480168C90512
:1072600011D40168821511430160FFF7FFFC009003
:1072700005E0FFF7FBFC0099401A642837D8454821
:107280000068C005F5D532680321090560680A4029
:107290000140914208D08103890F032904D131684C
:1072A000890301D50120F8BD2A69032109040A4098
:1072B00022D0084090421FD0207880061CD5286933
:1072C0002A6988430121C9040A432A612A698A4339
:1072D0002A612861C0050FD5FFF7C8FC009008E0BF
:1072E000FFF7C4FC0099411A2B48814201D90320C1
:1072F000F8BD28698005F3D561688803800F0328ED
:1073000005D132680005824301400A433260286992
:10731000032261681204114008432861002F04D041
:10732000B16B012000078143B1632078C00705D00D
:10733000E868A168800880000843E860207880073A
:1073400005D5E8680C218843E1680843E8602078A7
:10735000400706D5E868032189028843216908436C
:10736000E8602078000706D5E86803210903884310
:1073700061690843E8602078000606D5E8680321C3
:1073800089048843A1690843E8600020F8BD000033
:10739000401002400070004088130000F8B50E460F
:1073A000050038D05E480068C007C00FB04214D254
:1073B0005B4C20684008400030432060FFF756FCDB
:1073C000074605E0FFF752FCC11B564881427AD8B8
:1073D0002068C007C00FB042F4D12878524C800713
:1073E00005D5E068F0218843A9680843E060287863
:1073F000C00752D06868022806D0032807D0216849
:1074000001280AD0890504E02168890301E0216888
:107410008901002903DB0120F8BD4907F9E7E1688C
:10742000890889000143E160FFF720FC074668688E
:1074300002280AD0032814D001281ED029E0FFF723
:1074400015FCC11B374881423DD8E0680007800F1A
:107450000228F4D121E0FFF709FCC11B3148814229
:1074600031D8E0680007800F0328F4D115E0FFF75A
:10747000FDFBC11B2B48814225D8E0680007800F27
:107480000128F4D109E0FFF7F1FBC11B2548814237
:1074900019D8E0680007800FF5D121480168C907B5
:1074A000C90FB14217D90168490849003143016049
:1074B000FFF7DCFB074608E005E0FFF7D7FBC11B41
:1074C0001848814201D90320F8BD15480068C0075B
:1074D000C00FB042F1D12878400706D5E0680721F7
:1074E00009028843E9680843E0602878000707D567
:1074F000E0680721C90288432969C9000843E060A0
:1075000000F03AF8E168094A0906090F515CC840E1
:107510000749086007480068FFF7CAFBF8BD00008C
:10752000002002408813000000100240A2C300089F
:10753000840100207C010020044805490068C968D6
:10754000044A4905490F515CC84070478401002036
:1075500000100240BBC30008044805490068C96820
:10756000044A8904490F515CC840704784010020D7
:1075700000100240BBC3000870B51A4AD3681A490C
:107580000C2018408D0004280CD04E00082810D084
:107590000C2810D050680004410F0120C003491C82
:1075A000884070BD1068C00601D5084670BD2846E9
:1075B00070BD304670BD98020C4C000F205C1B0261
:1075C0009C0FD368641CDB0301D5314603E01268CD
:1075D000D20600D4294602F0DCFE22460023FDF745
:1075E0009DFD70BD0010024000093D00B2C30008BF
:1075F000FEB505007ED0FE4CE7680C20E66807402B
:107600000120000406402878C00747D0082F05D085
:107610000C2F0AD101200004864206D12068800385
:107620003CD568680028E5D038E00120696800048E
:10763000814203D121680143216011E00523012229
:107640001B0492049942216802D111432160F1E7A1
:1076500081432160216801400091206890432060AF
:10766000686800280DD0FFF701FB009005E0FFF7E8
:10767000FDFA0099401A64287BD820688003F6D56B
:107680000CE0FFF7F3FA009005E0FFF7EFFA00993E
:10769000401A6428F0D820688003F6D42878800740
:1076A00056D50923E868042F0DD00C2F01D1002EE8
:1076B00009D000283CD02168994301432160FFF79D
:1076C000D5FA064628E02168490701D5002891D05F
:1076D00061681F22120291432A69120211436160FC
:1076E0002168994301432160FFF746FFE1680906DD
:1076F0000A0F00E08BE1BF49895CC840BE490860C1
:10770000BE480068FFF7D4FA002873D120E0FFF7E5
:10771000ADFA801B0228AFD820684007F7D5606813
:107720001F210902884329690902084360600FE0AC
:107730002068400840002060FFF798FA064604E001
:10774000FFF794FA801B022896D820684007F7D4E8
:107750002878C00660D5002F0CD0A86900284AD030
:107760002068FF21013108432060FFF77FFA0646B9
:107770002EE0C1E02068800502D5A8690028A6D0C7
:107780006068072149038843296A0843606060688C
:10779000297F0002000A090608436060286A410B3D
:1077A0000120C003491C8840E16809060A0F91497D
:1077B000895CC8409049086090480068FFF778FAF3
:1077C000002817D128E0FFF751FA801B0228A2D821
:1077D00020688005F7D56068072149038843296A36
:1077E000084360606068297F0002000A09060843B8
:1077F000606011E0E2E02168FF20013081432160F8
:10780000FFF734FA064604E0FFF730FA801B02283F
:1078100072D820688005F7D42878794E000724D5DF
:1078200068690028306910D0012108433061FFF7F2
:107830001DFA009005E0FFF719FA0099401A022896
:107840005AD830698007F6D50FE040084000306113
:10785000FFF70CFA009005E0FFF708FA0099401ACC
:10786000022849D830698007F6D42878400766D5C1
:1078700000200290A06BC00006D4A06B0121090774
:107880000843A063012002905E480168C90511D435
:107890000168821511430160FFF7E8F9009005E0E7
:1078A000FFF7E4F90099401A642825D85548006884
:1078B000C005F5D5FF20AA680130824203D13169A5
:1078C0000143316111E001218902002A07D005231B
:1078D0001B029A4203D132690A433261EFE73269EF
:1078E00082433261306988433061A868002810D033
:1078F000FFF7BCF9009008E05FE0FFF7B7F9014639
:107900000098091A4048814257D830698005F4D55B
:107910000DE0FFF7ABF9009006E0FFF7A7F900993B
:10792000411A3948814248D830698005F5D4029817
:10793000002804D0A06B012109078843A063686A6E
:10794000002866D00C2F3ED001263606022820687B
:1079500005D0B0432060FFF789F905462FE0B0431A
:107960002060FFF783F9074604E0FFF77FF9C01BAB
:10797000022822D820688001F7D4E96AA86AE26860
:107980000843296BFD231B049A4311430843E0601D
:10799000206830432060FFF769F9054604E0FFF7EF
:1079A00065F9401B022808D820688001F7D530E02F
:1079B000FFF75CF9401B022801D90320FEBD2068B7
:1079C0008001F5D425E00128F8D0E0680121090400
:1079D000AA6A014091421AD10F218904EA6A014042
:1079E000914214D1032189050840296B88420DE09A
:1079F00000100240A2C30008840100207C01002086
:107A000040100240007000408813000001D00120A7
:107A1000FEBD0020FEBDF8B504000ED0FF27606A51
:107A20000537002500280AD02561656126464036C5
:107A3000A562707C002807D00AE00120F8BD6068CC
:107A4000B842F3D0E561F1E73574204600F03EF826
:107A5000022171742068026840239A430260212346
:107A6000A26860689B021A4038401043E3688A02AB
:107A70001340184323690B40217D1843C907C90FE0
:107A80000843A169931019400843E169382319405C
:107A90000843216A802319400843A16A93001940D2
:107AA000084321680860A0690421000C0840616A4D
:107AB000102319400843216848602068C169914338
:107AC000C1616565012070740020F8BD10B586B0F5
:107AD000044614216846FDF76AFB10492068884275
:107AE00019D10F48416B821411434163C16A0122CD
:107AF0001143C162C06A002110400590E02000904F
:107B00000220019003200390029104910520694610
:107B10000007FEF7DBFF06B010BD0000003001409B
:107B200000100240094910B5401E884201D90120C9
:107B300010BD074C60610321081F02F065FC0020A6
:107B4000A06107202061002010BD0000FFFFFF00A2
:107B500000E000E070B505462C46022020340029E4
:107B600008D004290BD008290ED0627F012A10D03A
:107B7000012070BDA27E012AFAD1A0760AE0E27E41
:107B8000012AF5D1E07605E0227F012AF0D12077A5
:107B900000E060770122286801F028FF01222868B0
:107BA00092070121904205D0074A904202D0074A2D
:107BB000904204D182685207520F062A02D002680E
:107BC0000A430260002070BD00080140001401401B
:107BD00070B504460D460068002201F007FF2068DA
:107BE000016A0C4A114203D1016849084900016049
:107BF00001202034002D06D0042D06D0082D06D0FB
:107C00006077002070BDA076FBE7E076F9E720778B
:107C1000F7E700001111000070477047704700003F
:107C2000F8B502680446D06911689668814B05462C
:107C30001D402023002D6CD0F7077F4DFF0FBC4661
:107C40000D402F4379D02546C7078035002F06D039
:107C5000CF0504D5012717622A683A432A608207B4
:107C600008D5F20706D0276802223A622A6804275C
:107C70003A432A60420708D5F20706D02668042254
:107C800032622A68022632432A6002070AD50A466F
:107C90001A406646324305D02668082232622E68B2
:107CA00016432E60020508D54A0106D50122266832
:107CB000D20232622A681A432A602A68002A30D027
:107CC000800606D5880604D5616E002901D02046BD
:107CD0008847286821688968490602D42821084213
:107CE00025D0204602F0A1F820688168490619D500
:107CF000826840218A438260206F002812D04F4959
:107D00008163206FFEF748FD00280AD0206F816B49
:107D100006E0850611D58D060FD5616E77E0204609
:107D20008847F8BD2046FFF779FFF8BD05E02046FB
:107D3000FFF774FF00202860F7E7256E012D56D16C
:107D4000C50654D5CD0652D5102616622068816826
:107D500025464906403500292ADA226F116849680C
:107D60000904090CE1D02F8B8F42DED96983116899
:107D70000968890617D401683201914301602068BF
:107D800081684908490081602068816840229143E8
:107D90008160E3670020206620680168B1430160CC
:107DA000206FFEF7D7FC288B698B401A81B21AE04E
:107DB000298B6A8B891A6A8B89B2002AB5D000296F
:107DC000B3D00268FF252135AA430260206882688B
:107DD000520852008260E3670020206660662068D7
:107DE0000268B24302602046FFF716FF9DE7C50216
:107DF00008D5750206D50120000510622046FFF760
:107E00000CFF92E7050605D50D0603D5A16E0029E6
:107E100085D18AE7400688D5480686D51168204670
:107E20004024A143116083670021816600F043F97B
:107E30007BE700000F08000020010004519D0008AE
:107E400010B5040003D0A06F002802D007E0012085
:107E500010BD002174200155204600F027F8242091
:107E6000A06720680168490849000160204602F0C7
:107E70002FF80128ECD0606A002802D0204601F0DB
:107E800051FE206841680922D20291434160206876
:107E900081682A2291438160206801680122114390
:107EA0000160204601F0A4FE10BD0000F0B587B0CF
:107EB000064614216846FDF77AF92C493068884255
:107EC00051D12B48416B0122920311434163C16A96
:107ED00001221143C162C06A0025104005900320B1
:107EE000400200900220032701A9A1C104200490B0
:107EF000052069460007FEF7E9FD1F4C1D48A560F7
:107F0000E56081C48027E560A7602020256160616D
:107F10000002A0611848083CFEF7B8FC002801D018
:107F2000FDF76AFF3467A662144C124821461438E4
:107F300020600320606010200831A1C16561A56147
:107F4000E56120462562FEF7A1FC002801D0FDF77F
:107F500053FFF466002201211B20A662FFF70EF9F1
:107F60001B20FFF7FFF807B0F0BD0000003801400C
:107F700000100240300002405017002098170020E7
:107F800070B5C36F202B27D100290BD0002A09D050
:107F9000012483682403A34206D10369002B03D183
:107FA000CB0701D0012070BD034660331C7D012C3E
:107FB00012D001241C7500230366084C0368A342F9
:107FC00007D05C68240204D51C680125AD062C434B
:107FD0001C6002F07DF870BD022070BD00480040BA
:107FE00070477047FFB50446806F83B017460D4653
:107FF00020285ED1002D0AD0002F08D0A168C00132
:10800000814207D12069002804D1E80702D001206D
:1080100007B0F0BD204660300090007D012848D0B8
:108020000098012101750020802108512120A067BE
:10803000FEF71CFE264640360190378277820120EB
:10804000A1680003814202D12069002805D02F4693
:10805000002500990020087511E00027F9E70022AB
:108060008021204602F07AF8002815D1002F15D083
:108070002168387888627F1C708A401E7082708AFE
:10808000019B002806980090E9D10022402120465B
:1080900002F064F8002808D00320B9E72888216896
:1080A000C005C00D8862AD1CE6E72020A067002057
:1080B000AEE70220ACE77047034D044C04A002F089
:1080C00047F9E560FAE700000400FA0500ED00E07A
:1080D000486172644661756C745F48616E646C657A
:1080E000722E0D0A0000000070B586B0142168469B
:1080F000FDF75DF801240B480C4EC4800A48A50228
:108100004483224629463046FEF7A9FD002102910C
:1081100003910095019469463046FEF7D7FC06B0FE
:1081200070BD0000280E00203C010020000400501B
:1081300010B505242407002204212046FEF78FFDF8
:10814000002208212046FEF78AFD0A2002F065FB86
:10815000012204212046FEF782FD0A2002F05DFB89
:10816000002204212046FEF77AFD10BD10B505243B
:108170002407002204212046FEF771FD0122082178
:108180002046FEF76CFD0A2002F047FB0122042185
:108190002046FEF764FD0A2002F03FFB0022042186
:1081A0002046FEF75CFD10BDF8B500240526074605
:1081B00025463607002204213046FEF750FD0A20EE
:1081C00002F02BFB012204213046FEF748FD600639
:1081D000040E08213046FEF735FD002801D0641C4E
:1081E000E4B2052002F019FB6D1CEDB2082DE1D3BD
:1081F000002F03D0FFF79CFF2046F8BDFFF7B6FF26
:10820000FAE770B5052605463607002204213046F8
:10821000FEF725FD0024E80901D0012200E000223C
:1082200008213046FEF71BFD6806050E0A2002F005
:10823000F4FA012204213046FEF711FD0A2002F073
:10824000ECFA002204213046FEF709FD0A2002F074
:10825000E4FA641CE4B2082CDDD370BD10B505242B
:108260002407012208212046FEF7F9FC01220421FF
:108270002046FEF7F4FC002208212046FEF7EFFC22
:108280000A2002F0CAFA002204212046FEF7E7FC89
:1082900010BD10B505242407002204212046FEF756
:1082A000DEFC002208212046FEF7D9FC0A2002F05D
:1082B000B4FA012204212046FEF7D1FC0122082154
:1082C0002046FEF7CCFC0A2002F0A7FA10BD70B5DC
:1082D00005252D070024012208212846FEF7BFFCB2
:1082E000062002F09AFA012204212846FEF7B7FC84
:1082F000062002F092FA07E0641CE4B2FA2C03D9DB
:10830000FFF7C7FF012070BD08212846FEF79AFC41
:108310000028F1D1002204212846FEF7A0FC00200D
:1083200070BD0000F8B501F095FC01F0C5FC5A489D
:108330000068C069FDF750FE584C5949A082898FEA
:10834000584E0025002931D0A26A730356499A423B
:1083500002DB02220A7000E00D700A780121890216
:10836000002A05D0012A0ED0022A10D0032A1DD1DE
:10837000608B01282CD0022818D1474808214038AA
:10838000FFF726FC12E0FF22F5329042F0D2608B1C
:1083900001281BD0022804D008E03046FEF75FFC1D
:1083A00004E03D4808214038FFF7D4FBFDF71EFFED
:1083B00020700121C9023046FEF744FC0127FF036B
:1083C00000282BD0A079002804D007E00022E4E7A1
:1083D0000122E2E70120A07101F022FF8021304656
:1083E000FEF730FC002806D0002208213046FEF7B8
:1083F00036FC012205E0012208213046FEF72FFC61
:108400000022052039460007FEF729FC244C274EA0
:108410004034A08C264F012803D01CE0A571002217
:10842000EAE724486946088072B680212248FDF7B1
:10843000FBFC002804D0022269461F48FDF798FD86
:1084400062B61EA001F084FFA58403F0BDFE642087
:1084500002F0DCF9FE60608C012808D110486584C8
:10846000058003F0B1FE642002F0D0F9FE60208C9C
:10847000012806D1258403F0A7FE642002F0C6F986
:10848000FE600748114A0188914202D1C088002845
:1084900000D1FE60F8BD0000CC1600203C01002099
:1084A000E80D002000040050840000200400FA05BC
:1084B00000ED00E0AAAA0000384A0008BDF8C8EBA9
:1084C000C9FDBCB6C4A3CABD0D0A0000AA55000070
:1084D00038B55721202000F07AF80321212000F040
:1084E00076F84021222000F072F80821232000F0C5
:1084F0006EF8AA21302000F06AF81048018F142984
:1085000001D8002901D1012101870C4C4034618838
:10851000142901D8002901D102216180008FC1B244
:10852000322000F054F8A178332000F050F868466B
:1085300000F006F80A2002F070F938BDE80D0020BE
:1085400010B501460F2000F021F8002800D00120CE
:1085500010BD10B50446FFF781FE3220FFF751FE33
:10856000FFF7B5FEE0B2FFF74CFEFFF7B0FEFFF7F6
:1085700075FE3320FFF745FEFFF7A9FE0020FFF749
:1085800013FE0446FFF785FE204610BD10B50C46CD
:10859000FFF7DFFF2070012010BD70B50D460446C7
:1085A000FFF75CFE3220FFF72CFEFFF790FEE0B2F3
:1085B000FFF727FEFFF78BFE2846FFF722FEFFF7A7
:1085C00086FEFFF766FE0A2002F027F970BD10B59F
:1085D000FFF7E3FF012010BD10B50248FEF781FC54
:1085E00010BD000004160020FEB50446002772B638
:1085F000334A01688B1804D13248C76803208004CD
:10860000074088680190C868009048698E69002B0F
:1086100008D12C4940398B6ACD042B438B628B6A7D
:10862000AB438B62014631433CD025492368CB42A2
:1086300005D12449CA6803239B049A43CA6025468E
:108640002035002810D021680A6901231A430A61E5
:10865000216848610821204600F036F8032800D13F
:10866000A873216808204860002E10D02068016996
:10867000012211430161206886611021204600F02B
:1086800023F8032800D1A8732168102048600C4803
:108690002168C14206D10B48C1680322920491436C
:1086A0003943C160206801694908490001612168B6
:1086B0000198886021680098C86062B6FEBD00001D
:1086C0000084FFBF4010024070B506460B480D46BF
:1086D000002409490068FCF70BFD7D21C9004843CF
:1086E0003168401E00D103240B682A469A4301D00A
:1086F0000028F6D1204670BD204E000084010020E5
:108700001CB5002116480091144A01910260C16312
:1087100012054260816007228263012202610246E3
:10872000C16020321170FF235170C23343628162F5
:10873000117301638161042241634261C161FDF7EC
:108740006FFE084800908013019069460448FDF7C9
:1087500017FE00210248FDF7BDFD1CBD00240140AD
:10876000A81500200200000408B50848016B01228A
:1087700011430163006B01211040009000220A2088
:10878000FEF7FCFC0A20FEF7EDFC08BD00100240DD
:10879000F0B587B014216846FCF709FD4748C26A66
:1087A00004210A43C262C26A0A400592C16A802655
:1087B0003143C162C16A31400591C16A012421433C
:1087C000C162C16A21400591C16A02252943C16283
:1087D000C06A22462840059005201C210007FEF7AC
:1087E0003EFA012236493748FEF739FA0022364967
:1087F0003448FEF734FA91210520002209020007CF
:10880000FEF72DFA314801900027052069460297AE
:1088100000940007FEF75AF90C20009011200190F7
:10882000032003900520029769460007FEF74EF9E2
:1088300010206A46039591C2052069460007FEF79D
:1088400045F91120019002976946039700941D484D
:10885000FEF73CF91E4801906946009502941948BC
:10886000FEF734F9E0020090694601970295154839
:10887000FEF72CF91748694691C1694611480397DC
:10888000FEF724F991200002694691C1052069464E
:1088900000070397FEF71AF969460A480197009600
:1088A0000294FEF713F9002201210520FEF766FC71
:1088B0000520FEF757FC07B0F0BD00000010024095
:1088C00001020000000400500830000000001110F8
:1088D000000021100832000010B50F4C0D48206038
:1088E000FF20053060600020A060E06020616061D2
:1088F000E0610121206249026062A161A06207205B
:10890000E0622046FFF787F82068016840221143A3
:10891000016010BD003001403416002000B585B064
:1089200014216846FCF743FC0E480D490160E12123
:108930004902416000218160C160016181610C22B6
:10894000C1614261016230214162012109038163F9
:108950004900C163FFF774FA01F05CFC05B000BD8B
:1089600000380140CC16002070470000F0B589B0F7
:108970000A2002F09DFC7D20400102F0B3FCFF4C78
:108980000025A570FE482066607C0C2801D30B20D2
:10899000607460790A2801D90A206071F948E5708D
:1089A000F94E00783071F949A07909784000084300
:1089B000A17D89000843F071E06BF070010A31720B
:1089C000401CE0636079B07442003046F0491330D7
:1089D000FCF7D4FB6079EE498200400080196031D9
:1089E0001330121DFCF7CAFB607906214200484390
:1089F0008019E8491730921CFCF7C0FB2E20205E3E
:108A0000002803D0E449098A0818E0856079DB4929
:108A1000C000223182190B7B53764B7B9376062262
:108A20007272DE4A1D301278B272A28C3273D64A4C
:108A30000B79133A1375497951750022D24902F026
:108A400021FD60790021C0001D3002F02DFDD448C9
:108A5000FEF722FB01272085BF0309E0D048FEF77F
:108A60001BFB80B22085E18EFF392D39884206DB61
:108A7000E18E80B28842F1D3C9198842EED8022033
:108A800002F066FCC0480126C571A574A573267462
:108A9000E573C348FEF700FB60850746E570607923
:108AA000FCF74CFEBF4AC04BFCF72CFD01F04AFE20
:108AB0000022BE4BFCF774FCFCF7A0FE0006C10CC4
:108AC000C81980B2F103A085884201D3401AA0855D
:108AD000B748E0642079401C2071B148FEF7DCFA09
:108AE0002085AB48A54F643840370690B1E1AC48CB
:108AF000FEF7D2FA20850BE0A948FEF7CDFA80B246
:108B00002085A18D884203D3AA4A8918884207D3B9
:108B100000210F2002F04CFBA74920640842EBD053
:108B2000206C411C1FD040047ED58122D20100213F
:108B30000F2002F07CFC0021102002F039FB4106DE
:108B40009348490E00227C38E16502F067FB002063
:108B500002F0C8FB002002F07AFB8D487C38417A95
:108B60000729C3D101E001F071FC02229349401DA5
:108B7000FCF728FB0028B9D102F0E7FCE167A06709
:108B800002F0D0FC7D4B803303C3E0788049401C69
:108B9000E07083390B7A68460370497A4170008827
:108BA0000390E18C88427DD1774985488C31C98E0C
:108BB0000180754971488C31098F41847848FEF7EE
:108BC0006BFA208502F006FA6C48FF2280300168BB
:108BD000406852040023891858410206080A1043CD
:108BE0004108490000900A0E080264498031CA60B9
:108BF00088606548E36F0A30A26F02F07BFC607901
:108C00008100614808185D49163080310CC902F0B6
:108C100071FC5A488030C36882685B48123002F0A9
:108C200069FC0821584800E006E14172B430C07C7C
:108C30000009607514D05648022260497738FCF765
:108C4000C1FA00280CD15048A674C671E06D504995
:108C50001638C2B26639C81DE274FB30FCF78EFAD2
:108C600060790022800048491C3002F00BFC6079DA
:108C7000002180001C3002F017FC009802F011FB6C
:108C8000012002F065FB207302214E48FDF7DAFF58
:108C900000281DD000213D4801703B498C31488E91
:108CA000049000E05AE03881888E78818446A06C78
:108CB000FF310531E0640860DC392065C97C0907B3
:108CC000090F032900D02175E16D1C2902D015E0A0
:108CD0000121E0E72C49294A8C31C98F1186069B76
:108CE0002C4A1B881380884207DD002805DD0029F7
:108CF00003D0207E401C207600E025762571A673E7
:108D00000498B8816046F881E673608C2E49FF3084
:108D1000C33080B2608488420CD9494240186084D4
:108D200027487D220188D200491C89B201809142E6
:108D300000D3058022487D210088C9004843618C0A
:108D40004018606500F078FD207B002805D10021E7
:108D50000F2002F02DFA0006F9D583E0FDF724F983
:108D60000B4A03219032115407498C314A8E3A81C3
:108D7000898E7981E26D1C2A2ED127E070000020B7
:108D80003F420F003C0100205C12002070010020D7
:108D90008C130020C8140020280E00204C01002055
:108DA00004160020B81E85EB51B8CE3F00000840E5
:108DB000A0860100983A000000D02724600100201E
:108DC0006C01002000040050E7030000614B4200EA
:108DD000D318069A12885A8080005F4B5E4AD43BB3
:108DE00002905D4982189B8F138030314118A26C2C
:108DF0004A605A4940185A4916300CC902F07AFBA9
:108E0000216EA06C884207DA534A02995158012911
:108E100002D12066039905914F49029A89588142EF
:108E200017DD012915DD2146002812DD0398C884CD
:108E30000220087065730CE04A4A00210F2002F0FE
:108E4000F6FA6079E178401C814202D0002002F0FD
:108E5000FEF9208DA18D884200D248E6424A891849
:108E60008842FAD8A07B012801D00220A07302F02A
:108E7000B1F83C4A00210F2002F0D9FA20790028ED
:108E800017D03A4909888A008A18824200D2257090
:108E9000002000F0E5F8A07C002839D02E496C3184
:108EA0000B78A372487860728A782272022B17D0EE
:108EB0002EE0E16C226E323920468A420EDAC17908
:108EC0002A4A491CC9B2C171128852008A42E2D2B0
:108ED0000599C184022101706573DCE7E571DAE769
:108EE00010280CD0C82813D2214BC91C1818FCF725
:108EF00045F903F069F9642001F088FC33E61D4D63
:108F000028684000000E03D1C878FCF7FCFB2860FD
:108F100000202378627B65790FE00F4E4100303EE0
:108F2000775A1836765AB74205D00B4F02230022E3
:108F30000126483F7E52401CC0B2A842EDD32370A8
:108F40006273084A002180320F2002F070FA09B0E3
:108F5000F0BD0000C8140020BC1300205C120020EB
:108F6000F000002000D02724983A00004C01002097
:108F7000E80D002064010020F8B52E4C0546E06E97
:108F80002D4A281A411E2067914215D21A21615E8E
:108F9000081AFCF7BFFB294A294BFCF7B3FA06462F
:108FA00032200F46205EFCF7B5FB32463B46FCF70D
:108FB000F7F9FCF7FFFB6086002060761D481C2354
:108FC000C35E828C1F48008884461F4806881DE0C7
:108FD0006046484380181D4F80B238803027784360
:108FE0006427643078431A4F6066C01985420BD2FB
:108FF000C8B2184932220880606EA25E411BC918AF
:109000008918A166E066F8BD491C6176617EB142AF
:10901000DED33020424310486421101848430F49E2
:109020004118E16660663221401B615EC01840183D
:10903000A066F8BD70000020CF0700009A999999AA
:109040009999B93F5A0100204C0100206E0100207F
:1090500078ECFFFF5801002074270000C0BDF0FF2E
:10906000FEB5294D2988491C8FB228492F800E88CA
:10907000FCF750FB264A274BFCF744FA019100907D
:1090800025483146FCF734F8244C218F4218B7426A
:1090900006D3002028802248019E1018009D02E07F
:1090A0001046019E009DFCF749FB33462A46FCF71B
:1090B00077F9FCF7A3FBA086012580B2ED03A84257
:1090C00001D3401BA086E08BFCF738FB154A164BFA
:1090D000FCF780FA0646A08E0F460090FCF72EFBA8
:1090E00032463B46FCF75CF9FCF788FB80B2E08631
:1090F000A84201D3401BE0860C49009809684861EA
:1091000000982087FEBD0000580100204C0100207F
:109110001904560E2D624040E17A000070000020D4
:109120001F050000F853E3A59B843E400416002071
:1091300070470000F0B589B0002004900A2002F0CA
:10914000B7F87D20400102F0CDF8B34800228270CC
:10915000C16BB34C491CC163B049C38D098A254614
:10916000C918C1852146C275133107914731039152
:109170006D393135AB4F223005910290A64E0F214B
:10918000A948717100782071A84AB079127840001E
:109190001043B27D92001043E071B08FE070000A7E
:1091A0002072A17431461E229C310798FBF7E6FF1E
:1091B000402228469E49FBF7E1FF029903980A7B6B
:1091C000C274497B0175092060729A480078A072C8
:1091D000B08C2073F07D410030469C300918059812
:1091E0000A78027549784175762000228C4902F090
:1091F00049F970790621484300211C3002F054F9E6
:10920000022002F0A5F800210F2001F0D1FF384222
:109210003064F8D0306C411C18D040047ED58122D7
:10922000D20100210F2002F002F90021102001F0EC
:10923000BFFF41067A48490E0022B43001F0EEFF2C
:109240007748B430417A022902D0BDE001F0FEF83F
:1092500002227949401DFBF7B5FF0028F5D16E4881
:109260000222C07D41006C489C3009186C48B53022
:10927000FBF7A8FF0028E8D102F067F9664AD1673A
:10928000906702F04FF9644A803203C204980028C4
:109290002CD1012004906248684E8C30C08E604909
:1092A00030805D488C31098F41846548FDF7F4FEBC
:1092B0005949644A0885488CFF30C33080B24884DD
:1092C00090420CD952428018488430885D4A401C34
:1092D00080B20B323080904201D300203080308841
:1092E0007D22D20050434A8C801848654C4869461C
:1092F0008C30428E0A80808E488049490422B531E4
:10930000C81FFF38FBF73AFF4348494AC07D009920
:10931000800011504049803103C900E075E0FF230F
:109320005B040022C01851410906060A0E4330466C
:1093300001F0B7FF710849000A0E080236490026FD
:109340008031CA6088603448C36F826F34484838BF
:1093500002F0D0F8304880300CC83148443802F070
:10936000C9F82D488030C36882682D48403802F023
:10937000C1F82B49002252393C2002F083F8002129
:109380003C2002F091F8012001F0E2FF224908732D
:1093900008468078401C887001210520C903000719
:1093A000FCF716FE1C48007B002805D100210F2089
:1093B00001F0FEFE0006F9D5802200210F2002F008
:1093C00036F81548467002E01349012048701248EB
:1093D000C17D491CC9B2C1750F2900D2CEE60498DF
:1093E000002810D10C4A1849908C002802D00B8814
:1093F000984201D908889084144980B20988401E97
:1094000048431349088009B0F0BD124A00210F20DB
:1094100002F00DF8D8E7000070000020280E0020B0
:109420005C12002000D027243C01002070010020A5
:10943000781400204C010020600100206C01002005
:1094400004160020E7030000480100204601002028
:109450004401002000902724F8B531492F480860C6
:1094600002F056F92F4800F0A7F92F4CE0822D4862
:10947000801C00F0A1F920832A48001D00F09CF90F
:1094800060832B4829494180014640310979294FA1
:109490000906090E617006D1C7800121C1870A2122
:1094A000418700218187244AC18E1170C18F2171AB
:1094B000818F6171817AA1708588052165626181E2
:1094C000C6883046FBF714FEA08101462846FBF70C
:1094D0000FFE8800081885B2164825816843FCF7FE
:1094E0002DF9164A164BFCF775F8FCF787F9E08161
:1094F000658231463846FBF7FBFD20820146C820D5
:10950000FBF7F6FDE0830120A083FCF765FDA08258
:10951000E2890C490C48FDF7C3FDF8BD41A20008E3
:1095200068000020004F00083C0100202E020000CF
:10953000E80D0020E803000018000020F853E3A520
:109540009B843E40FF7F000004160020F8B5774C56
:1095500000202071764E01203080764FC820388060
:10956000E07A401CE072C00706D0A08C411EA184A6
:10957000022801D2C820A0840120C043FFF770FD5B
:109580000A2001F095FE7D20400101F0ABFE022192
:109590006948FDF757FB00283FD00020674980004D
:1095A0000978684D49000843654909780843A8725D
:1095B000102068726448C1887D20C000FBF798FDC8
:1095C0006873624860490078A87328460B308A782F
:1095D0000270C97841705C49421C20310B7ED37007
:1095E000497E11715849D01C22310B7E5371497E3E
:1095F0009171554940310A7C0271497C41710022C8
:109600002946172001F03EFF0021172001F04CFFF2
:10961000022001F09DFE4E4D03E00120BEE7FEF763
:1096200081FE00210F2001F0C3FD28422064F6D006
:10963000206C411C77D0400473D58122D2010021D7
:109640000F2001F0F4FE0021102001F0B1FD4106D1
:109650003C48490E0022B430E16501F0DFFD394D90
:10966000B435687A11285CD102223A49681DFBF7AB
:10967000A9FD002855D1E81F027A69460A70407A90
:109680004870A97A3180C820FBF732FD3880287BEA
:10969000A0842846304F2838C08E38802946234879
:1096A0002839098F41842D48FDF7F6FC2085608C10
:1096B0002B49FF30C33080B2608488420CD94942C4
:1096C0004018608438882649401C80B20B313880AD
:1096D000884201D30020388038887D21C900484362
:1096E000618C4018606500F0A7F868460088E08447
:1096F000A87C14496071C731420008460D466930A4
:10970000FBF73CFD6079294642001648FBF736FD21
:10971000A18C0320FF2900D020703188322900D18C
:109720002070F8BDFFE700F091FE000070000020FF
:109730004C0100205A01002000040050400100208C
:10974000410100205C120020E80D002018000020DC
:1097500000D02724600100206C01002004160020A6
:10976000E7030000A413002070B586B014216846FA
:10977000FBF71DFD01250F4EED0300222946304663
:10978000FDF76DFA012000240190029469460095CE
:1097900003943046FDF79AF903200190029469463C
:1097A000009503943046FDF791F9022001F02EF860
:1097B00006B070BD0004005000887047704700007C
:1097C000F8B5044600206A461080194D55222A70CB
:1097D000AA226A700322AA70661DEE702A7169714E
:1097E000144A49008918AC712246E81DFBF7C6FCF3
:1097F000002007E029186A468978128889186A4685
:109800001180401CB042F5DB611DA81CFCF742FA38
:1098100001466846018029190078C8716846407879
:10982000087221460931024800F020FBF8BD000013
:1098300042150020E80D0020FEB5FFF79DFB2548EE
:10984000FDF72AFC244C86B2268560790A21081A85
:10985000C000FBF75FFF07460191A06EFBF76EFFAC
:109860001E4A1F4BFBF7B6FE00900D463046FBF735
:1098700065FF2B46009AFBF793FD3A46019BFBF7E9
:109880008FFDFBF7BBFF85B2A586E08BFBF756FF8C
:10989000124A134BFBF79EFE06460F462846FBF77F
:1098A0004DFF32463B46FBF77BFDFBF7A7FF81B23E
:1098B0000120C003E186814201D3091AE186854275
:1098C00001D3281AA0860349A08E09684861208721
:1098D000FEBD00000416002070000020F853E3A530
:1098E0009B843E40034A1168382389B2994301435F
:1098F000116070470030014010B5FDF7BDF910BD93
:1099000010B59AB034216846FBF751FC14210DA81C
:10991000FBF74DFC1C2112A8FBF749FC1B48016812
:109920000324E402A143C21489180160FDF732FC4C
:1099300017480169A143016106200090FF20013012
:10994000029001200390102004900220099040040E
:109950000B90000100240C900A946846FDF748FE25
:109960000F200D9003200E900F941094012111945C
:109970000DA8FDF713FD812012900320800418909C
:10998000149412A8FDF758FC1AB010BD00700040E6
:109990004010024010480168821511430160C168FF
:1099A0000E4A1140C16001680D4A11400160816892
:1099B00049084900816001680122920491430160D5
:1099C000C168FD2212049143C16000210161064972
:1099D0000448886070470000001002400C40FF8877
:1099E000F6FFF6FE0050000800ED00E010B5CB06D3
:1099F000DB0E0121046A99408C430462016A9A409B
:109A00001143016210BD0000F8B5102405252D0793
:109A1000AC62AF20800000F000FFAC6101F0DCFB25
:109A2000344C354F354E60670EE001F0D5FB606772
:109A3000FEF778FC606C411C6164142804D930A0E6
:109A400000F086FC3248C760606FB042EDD100265E
:109A5000666420780127FF03030000F0B2FC0504D0
:109A60000C192D3A3C00012239462846FDF7F7F83B
:109A7000FFF76CFD06E0012239462846FDF7EFF8B6
:109A8000FFF758FB002239462846FDF7E8F822E0A8
:109A9000607B0122401C607339462846FDF7DFF8E1
:109AA000FCF7B6FA002239462846FDF7D8F8607B65
:109AB000052810D926700EE0FEF758FFFCF74AFB88
:109AC000154814490068FBF7E3FBFBF745FEE0850A
:109AD00001E0FFF72FFB02211048FDF7B3F8002843
:109AE00005D000200E49087001F05CFAF8BD012095
:109AF000F8E70000700000200400FA053001CADE1B
:109B00004457204944204552524F522E0D0A00001E
:109B100000ED00E00000C8420000002000040050FA
:109B20007001002010B5818CC90707D001684A6810
:109B300001235B049A43836A1A434A60818C890734
:109B400007D501684A6801231B049A43C36A1A4374
:109B50004A60818C490707D501684A6801239B0444
:109B60009A43036B1A434A60818C090707D5016841
:109B70004A680123DB039A43436B1A434A60818C92
:109B8000C90607D50268916801231B039943836BBB
:109B900019439160818C890607D501688A68012381
:109BA0005B039A43C36B1A438A60818C490612D5C2
:109BB00003685A6801210905046C8A4322435A60EC
:109BC000026C8A4207D10268516803235B059943FE
:109BD000436C19435160818C090607D501684A68B6
:109BE0000123DB04806C9A4302434A6010BD0000ED
:109BF000F8B50446002680300660FDF737F80546C4
:109C000020680068124F000709D501212B46002269
:109C100049052046009700F0A1FA00280DD12068E0
:109C2000006840070BD501212B46002289052046FC
:109C3000009700F093FA002801D00320F8BD2020FF
:109C4000A067E0672666603426750020F8BD000036
:109C5000FFFFFF01F8B5154CC826E078002823D196
:109C60006079002820D101206071114D686B0027B8
:109C7000002818D0686BC821081A0FE00D48E16869
:109C8000405C61698847E068401CE060E068C82883
:109C900000DBE760696BC820401A761EE1688142EC
:109CA00001D0002EEADC6771F8BD000054000020EE
:109CB00000000240200D002070B5224CE078002802
:109CC0003FD1207900283CD1012020711E4EF1693E
:109CD00000250906002933DA2156625791420AD13C
:109CE000F06940062CD5A079002829D0A5712089DB
:109CF000401C208124E0A179002903D1A0710A2011
:109D000000F08BFD00202056CC2148430F4942181B
:109D1000206912181279B262401C00222061A256FA
:109D2000CC235A43895881420ADC25612078401CA3
:109D3000207020780E2800D12570A078401CA070DB
:109D4000257170BD5400002000380140F80100204A
:109D500010B5806A0022014640314A834A82FDF7ED
:109D60005DFF10BD70B5846AA06FE56F21688968DA
:109D700000260906002906DA212804D152200653BC
:109D8000204600F06BF820688068400606D5222D3A
:109D900004D15A200653204600F047F82046803070
:109DA00001681022114301602046FDF737FF70BDA6
:109DB00010B501460968806A096889061CD400222A
:109DC0005A210A5201680A68FF2301339A430A6044
:109DD00001688A68520852008A6001688A684023D4
:109DE0009A438A602021C167016E012904D101686C
:109DF0000A6810239A430A60016E012902D0FEF717
:109E0000EFF810BD5821095AFDF706FF10BD10B537
:109E1000806A016E012902D0FEF7E3F810BD5821D7
:109E2000095A4908FDF7F8FE10BD01680A68FF23CA
:109E300021339A430A6001688A68520852008A6096
:109E4000016E012904D101680A6810239A430A604F
:109E50002021C167002101664166704701680A68D8
:109E6000C0239A430A6020218167704770B5164C61
:109E7000E278002A0CD12279002A09D10122E2706D
:109E80000025C82903DC0222A256002A01DCE57065
:109E900070BD0123E356CC2253430C4AD150012319
:109EA000E356CC2673439B180A460146181DFBF760
:109EB00065F96078401C607060780E2800D165708C
:109EC000A078401EA070E2E754000020F8010020B6
:109ED000F8B50446016880682369E6691843636938
:109EE000002533431843724A0B68724E33400343D4
:109EF0000B602168486803231B039843E3681843F9
:109F000048602168A069914201D0236A18438B6898
:109F10000B263602B34303438B60674923686748C7
:109F20008B420CD1C0688007800F06D0012839D041
:109F3000022835D0032821D11EE001271FE0604907
:109F40008B420AD1C0680C21084027D0042829D0B0
:109F5000082825D00C2811D10EE093420ED1C168FB
:109F600003208002014019D001208002091A19D073
:109F7000091A15D0814201D1082700E010274F4966
:109F8000504840398600934232D1002F0CD0022F26
:109F90000DD0042F10D0082F7FD126E00027EEE748
:109FA0000227ECE70427EAE7FDF7C6FA06E00968AE
:109FB000C90605D4304603E0FDF7DEFA002872D06A
:109FC000626851005118814267D81103814264D3FD
:109FD000010E06025008002330185941FBF79EF885
:109FE00003210902411A384A55E00120C003E7E77E
:109FF0000122E369D20393422BD13B0000F0E1F947
:10A000000906090C4D114D4D4D274D00FDF794FAF1
:10A0100009E0FDF7A1FA06E00968C90605D4304653
:10A0200003E0FDF7A9FA00283DD0616840004A0826
:10A030008018FBF75DF880B20146244A103991423E
:10A040002BD8511C01400007400F084329E010465F
:10A05000EBE73B0000F0B5F90906090C21122121BC
:10A0600021232100FDF768FA0AE0FDF775FA07E001
:10A070000968C90606D4304604E00EE0FDF77CFA14
:10A08000002810D061684A081018FBF731F880B238
:10A0900001460E4A1039914203D9012503E01046CA
:10A0A000F0E72168C86000206066A0662846F8BD19
:10A0B00000480040F369FFEF0038014040100240C3
:10A0C0000044004000093D00FFFC0F00EFFF0000CE
:10A0D000F8B50446416540300026274602838037A4
:10A0E0003E602220E0672546206F603500281CD0A6
:10A0F0001749C162216F17480863216F16484863EA
:10A10000206F8663236F606D9C461346216802466C
:10A1100060462431FCF702FC002806D0102038608D
:10A120002E752020A0670120F8BD2E7520680168DB
:10A13000FF2201321143016020688168012211432E
:10A140008160206881684022114381600020F8BD51
:10A15000B19D00080F9E0008659D0008FFB581B005
:10A1600005460F46044660350A9E39E0701C37D01C
:10A17000FCF77CFD0499401AB04222D8002E20D072
:10A180002068016849072BD5C069C043000527D462
:10A1900001202168C002086220680168FF22A13204
:10A1A000914301602068816849084900816020204E
:10A1B000A067E0678034206000202875032005B088
:10A1C000F0BD20680168FF22A13291430160206840
:10A1D00081684908490081602020A067E067EBE7BB
:10A1E0002068C1693846884305D000210398814220
:10A1F000BCD00020E3E70121F8E7000010B50449D6
:10A200001020096808620248FDF70AFD10BD000031
:10A21000CC16002001490D208870704754000020A2
:10A2200010B5FEF7A1FAFEF779FBC82202490348F0
:10A23000FDF7A6FE10BD0000200D0020CC1600206A
:10A24000F8B53E4C002321783D4A1D46082910D020
:10A25000072947D0062950D0052952D0042953D0C8
:10A26000032954D0002956D0012958D002295AD0A8
:10A270005BE0A17800264A1F04E0314FBF5DFB1868
:10A280009BB2761C9642F8DB667927799A195118A9
:10A29000E3786278C9188918C9194018C0430006C4
:10A2A000000E1AD1012E14D0022E16D125482449B1
:10A2B000C018FAF763FF01F087FF642000F0A6FAE8
:10A2C000BFF34F8F21492048C860BFF34F8F00BFB5
:10A2D000FDE759081046FFF773FA2570E570A57081
:10A2E000A571F8BDA1795054491CC8B2A071A178DC
:10A2F000491F8842F5D1082001E0607007202070D6
:10A30000F8BDE0700620FAE760710520F7E7A0705D
:10A31000E5700420F3E7552807D10120EFE7AA28CC
:10A3200003D10220EBE7032803D02570E570A57068
:10A33000F8BD032020702071F8BD0000340100201A
:10A34000DE140020E80D00200400FA0500ED00E016
:10A3500010B5024A024900F0E5F910BD0DB500083C
:10A36000880100202021020C01D010211046020A91
:10A3700001D010460839020901D01046091F820891
:10A3800001D01046891E420801D0881E7047081A65
:10A390007047F8B5040C8BB2264682B25E430D0CB2
:10A3A0001046370C5843360480190021794116466F
:10A3B0006E43370C36048019794126466E4389195D
:10A3C000F8BD30B47446641E2578641CAB4200D2DC
:10A3D0001D46635D5B00E31830BC18474900CA02A4
:10A3E0000243100000D004204A0D01D00122104386
:10A3F000044A490D914201D102210843012800D1AC
:10A4000005207047FF0700008307FF22DB0E9A40FC
:10A410008907090E9940002808DB830809489B003A
:10A420001B18186890430843186070470007000F16
:10A430000838830804489B001B18D86990430843D8
:10A44000D861704700E400E000ED00E0BFF34F8FFB
:10A4500004490348C860BFF34F8F00BFFDE7000009
:10A460000400FA0500ED00E0F8B504464F1EC800F0
:10A470000838211815461E46086849683A460623DA
:10A480009A4310D02A463346FBF73CF83A46D200AE
:10A49000083AA3181A687F1E5B68FAF781FF062244
:10A4A0003B469343EED1022F23D0042F11D0062F29
:10A4B0002FD12A463346FBF725F8E36AA26AFAF75A
:10A4C0006FFF2A463346FBF71DF8636A226AFAF7E4
:10A4D00067FF2A463346FBF715F8E369A269FAF7E6
:10A4E0005FFF2A463346FBF70DF863692269FAF7E6
:10A4F00057FF2A463346FBF705F8E368A268FAF7E8
:10A500004FFF2A463346FAF7FDFF63682268FAF7E1
:10A5100047FFF8BD002210B5134610460149FBF76E
:10A5200059F810BD0000F03F10B5FAF739FF10BD23
:10A53000002210B5134610461146FBF74BF810BD2C
:10A5400010B50721024A00200907FBF7BBF810BD30
:10A5500001030000034A10B500201107FBF7B2F811
:10A5600010BD000001FDFFFF02E008C8121F08C176
:10A57000002AFAD170477047002001E001C1121F84
:10A58000002AFBD1704700000149086070470000B5
:10A590008C01002008B50021684601706B4601223D
:10A5A00002212C2000F052FF0221684601706B4608
:10A5B00001222C2000F04AFF08BD000038B50446F7
:10A5C0006D20694608706B46012207492E2000F075
:10A5D0003DFF0649002C01D0054A00E0054A2E2027
:10A5E00000F01AFF38BD0000060800000618000041
:10A5F000070600000716000038B504466B46022225
:10A600000021362000F0EEFDB3212300FFF7D9FE34
:10A610000E0F08153A3A3A3A1C273A3A2F34483A7C
:10A6200000216846017040784108490014E06946FD
:10A63000087880088000401C04E06946087880089B
:10A640008000801C08701DE0684602780A4048328D
:10A6500002704178802001436846417012E06846EC
:10A6600002780A40027040784106490EF4E76946D4
:10A6700048780221084303E069464878FD210840F4
:10A68000694648706B4601220021362000F0DEFE4C
:10A69000012200AB11463620013300F0D7FE38BD51
:10A6A00069460878CF21084069462030CAE708B5D6
:10A6B000032168464170012101706B46022200218E
:10A6C000362000F0C3FE0122D20306212D2000F027
:10A6D000A3FE012000F09AF80120FFF78DFF08BDCE
:10A6E00008B5020A69464A7008706B4602220421C6
:10A6F0002D2000F0ABFE0320694608706B46012256
:10A7000006212D2000F0A2FE0020694608706B464D
:10A71000012206212D2000F099FE0A212D2000F0B3
:10A7200047FD08BDF8B516460F460446002503E070
:10A730003946B047641C6D1C20780028F8D12846A3
:10A74000F8BD0000F8B54A002B4B520DD6182B4A25
:10A750000C460546142E2BDA002E12DA284BFAF797
:10A760001FFE00221346FBF78FF840D2002C03DABD
:10A770000124E40700253AE02046284337D0214C45
:10A7800014E0214F0B46F7403B402B4331D01C4B8C
:10A79000FAF706FE00221346FBF776F827D2002CC4
:10A7A00003DD01200005F0400419BC4300251EE034
:10A7B000332E1EDC33460027143BFF43DF40384274
:10A7C00017D00F4BFAF796FE00221346FBF75CF802
:10A7D0000DD2002C0ADD142E0CD03420811B012058
:10A7E00088404019A84200D2641C0546BD4321465A
:10A7F0002846F8BD641CF9E701FCFFFF9C75008842
:10A800003CE4377E0000F03FFFFF0F007D2110B5D4
:10A81000C900484300F001F810BD002140E000BF2E
:10A8200000BF00BF00BF00BF00BF00BF00BF00BF30
:10A8300000BF00BF00BF00BF00BF00BF00BF00BF20
:10A8400000BF00BF00BF00BF00BF00BF00BF00BF10
:10A8500000BF00BF00BF00BF00BF00BF00BF00BF00
:10A8600000BF00BF00BF00BF00BF00BF00BF00BFF0
:10A8700000BF00BF00BF00BF00BF00BF00BF00BFE0
:10A8800000BF00BF00BF00BF00BF00BF00BF00BFD0
:10A8900000BF00BF00BF00BF00BF00BF00BF491C1A
:10A8A0008142BCD37047FFB581B01E460F460400FD
:10A8B00026D00B9903980143A06A39438268072088
:10A8C0009047002818DB0A99A06A31438268062065
:10A8D0009047002810DB25462035A979032F01D9A0
:10A8E00008200143032E01D904200143A06A826895
:10A8F00009209047002806DA0120C04305B0F0BDCA
:10A900000020C043FAE7384600F000F920603046E6
:10A9100000F0FCF860600A9868700398A870EF7007
:10A920002E710B9868710020E8E70000F7B5044627
:10A93000002090B000900190002C05D06A460621BE
:10A9400001F07CFC062803DA0020C04313B0F0BD00
:10A950006846407801026846007800040918684695
:10A9600080780818FAF7EAFE0546684603910079F0
:10A9700001026846C0780004091868464079081842
:10A98000FAF7DCFE032206460F4692075C4BFAF705
:10A990007BFF07D200225B4B30463946FAF7A4FD15
:10A9A00006460F4603229207554B28460399FAF7AD
:10A9B0006BFF07D20022534B28460399FAF794FD08
:10A9C000054603912068FAF7B9FE02460B46304669
:10A9D0003946FAF7FFFD07460A200791205EFAF78D
:10A9E00099FE3A46079BFAF78DFD06460820099125
:10A9F000205EFAF77DFE0021C943FAF7C4FCFAF79E
:10AA00001BFF3246099BFAF7CBFC06910890606861
:10AA1000FAF794FE02460B4628460399FAF7DAFD48
:10AA200005461A200E46205EFAF774FE2A46334683
:10AA3000FAF768FD0C9009911620205EFAF76AFE7D
:10AA4000099B0C9AFAF7ACFC05910A902A4633460A
:10AA500038460799FAF756FD059B0A9AFAF752FD10
:10AA600005910A901420205EFAF754FE3A46079B9F
:10AA7000FAF748FD07461C200791205EFAF74AFEC8
:10AA80002A463346FAF73EFD0E900B911820205EC1
:10AA9000FAF740FE0B9B0E9AFAF782FC2A463346E1
:10AAA000FAF730FD0B910E902069FAF733FE0B9BFD
:10AAB0000E9AFAF775FC2A463346FAF723FD054647
:10AAC0000E46E068FAF726FE2A463346FAF768FC97
:10AAD0003A46079BFAF764FC059B0A9AFAF760FC72
:10AAE00001229207084BFAF70DFD02460B46129C15
:10AAF0000898069903C411980CC0002026E70000AE
:10AB0000FFFF5F4100007041E17A843F00B5012101
:10AB1000C9040300FFF755FC081A05080B0E1114B1
:10AB2000171A0320C00400BD0720C00400BD0F2079
:10AB3000C00400BD1F20400300BD3F20400300BDF6
:10AB40007F20400300BDFF20400300BD084600BD3C
:10AB5000FEB5264F0D4604000FD0002D0DD0264621
:10AB600000202036B071F07129680D208847002838
:10AB700001DA7800FEBD102801D03846FEBDA5627E
:10AB8000E968002901D028208847204600F030F8E5
:10AB90000028F3DBA06AA52182680E209047A06AF6
:10ABA000962182680F209047A06A02218268622065
:10ABB0009047A06A002182680E209047A06A002179
:10ABC00082680F2090477179302001910090062310
:10ABD000202201212046FFF766FE0028CEDB20461A
:10ABE00000F0AEF80028C9DB0020FEBDFFFFFFFF2C
:10ABF00010B586B0044614216846FAF7D8FA002C3E
:10AC00007ED0A06A122143686A4610209847122815
:10AC100077D1684600780122010168464078120326
:10AC20000009081843492081884201DD801A2081EB
:10AC30006846837840780007000D181860818842C4
:10AC400001DD801A608168460079012201016846B1
:10AC5000C0781205000309186846407900090818F1
:10AC60003549E060884201DD801AE060684640793D
:10AC70000007030B6846807900021B186846C079FC
:10AC800018182061884201DD801A20616846417AE7
:10AC9000007A0002081802B2284801210904A282A1
:10ACA000824201DD521AA2826A46D37A927A120255
:10ACB0009A1812B2E282824201DD521AE2826A4698
:10ACC000537B127B12029A1812B22283824201DD58
:10ACD000521A22836A46D37B927B12029A1812B2CE
:10ACE0006283824201DD521A62836A46537C127C7F
:10ACF00012029A1812B2A283824204DD501A01E0B5
:10AD00000BE008E0A083A06A01682820884700289B
:10AD100006DA0120C04306B010BD0020C043FAE7A8
:10AD2000C011C0072034002800D0802060710020AE
:10AD3000F1E70000FF070000FFFF0700FF7F0000B2
:10AD400010B5040009D0A06A072182680820904746
:10AD5000002805DA0120C04310BD0020C04310BD0B
:10AD6000072020342070002010BD0000FEB50446EE
:10AD70000020019000906079734940000E5A61787C
:10AD80002578491E7148CFB20163042D77D0072D75
:10AD900075D000210291217801736C49E379012279
:10ADA00092058969002B6CD0914381616748217AB3
:10ADB0004173217A82698907890B0A4382610021E4
:10ADC000042000F034FB324661492E2000F024FBC1
:10ADD0003846FFF7F3FB5F4E0522705D8100401897
:10ADE0005D49431807212B2000F030FB5B49029896
:10ADF00001220B180B21282000F028FB705D584918
:10AE000080000A580C21282000F011FBE0795549F8
:10AE100080004018A1794900425A0221272000F001
:10AE2000FBFA51487E00825B0421272000F0F4FAEF
:10AE3000E079002829D0A07804282CD02820694661
:10AE4000087220220621272000F0E6FA02AB012238
:10AE50002621272000F0FAFA444938014018E17809
:10AE6000890042580821272000F0E1FAA17A601CED
:10AE7000627A0902114313D016E000E001E00121DB
:10AE800088E71143F608816190E7642206212720B4
:10AE900000F0C2FAE0E71020694608720246D1E7E6
:10AEA00033490172090A4172417A007A0A02024367
:10AEB0002021272000F0B0FA2E4F0C2123203A68E1
:10AEC00000F0B5FAF01982880421232000F0A4FADA
:10AED000A07900280BD0E0792749012243180021EE
:10AEE000212000F0B3FA03200190012000902A07EE
:10AEF000120F10010243607800218007000B02430B
:10AF00000198000502430098400402432079C006DE
:10AF1000400902436079C00602431F2000F087FA0F
:10AF2000A07861780123084302040848DB0302612A
:10AF3000E179490319430A4302610021082000F026
:10AF400076FA0020FEBD000070C30008BC0100209E
:10AF50000428000018C3000824000020420000203C
:10AF600020C3000840C300084CC3000850C30008B9
:10AF70004110000038C300084400002038B50C46DA
:10AF800007498A8B002102432C2000F045FA6846CD
:10AF900004706B46012206212C2000F057FA38BDC0
:10AFA000BC01002010B5FFF7F5FA10BD10B504463E
:10AFB0000421362000F0FCF80121C902002C01D048
:10AFC000084300E0884302460421362000F02FFAAF
:10AFD00010BD000038B540206946087000210E20E1
:10AFE00000F0E6F80446002211460E2000F01FFA99
:10AFF0006B46012200210D2000F028FA074A0021AB
:10B000000F2000F014FA00F0EDF9224600210E2086
:10B0100000F00DFA02480021017338BDF8FF272423
:10B02000DC010020FEB50546042069460870514C3D
:10B030000020607521462031206348710873A08389
:10B040006063A06300F0C8F84B4E206002E000F09F
:10B05000C3F82060B042FAD10020FFF7CDFA00F02B
:10B06000BBF8464E20603078242801D9243806E009
:10B070000621FAF73DF80622101A4001084302069D
:10B0800001040A4301020A430243B26070600021D6
:10B090001E2000F0CCF900F09FF820606B460122E2
:10B0A0000021242000F0D2F91E20FFF719FB86B200
:10B0B000300AA0730420FFF713FB074600F08CF85A
:10B0C00020603806000E0DD002206946087101ABE1
:10B0D000012212212D2000F0B9F9A08B01210903D2
:10B0E0000843A08300F078F820600620FFF7F8FA04
:10B0F00060600720FFF7F4FAA060F006C00E20752C
:10B1000001D110202075C0B200F0DCF9E80707D0AB
:10B11000FFF7CDFAA08B0121C9020843A0830AE002
:10B120000521362000F02EF8154908400246052179
:10B13000362000F071F90120FFF75EFA00210420AB
:10B1400000F036F8A0610021262000F031F815212A
:10B150008903084302460021262000F068F90022F6
:10B160002621362000F058F900F036F82060002043
:10B17000FEBD0000BC0100203001CADE1800002026
:10B18000FFFD000038B5094C89B280B26B4602223F
:10B1900000F028F8002806D1684640780102684689
:10B1A0000078081884B2204638BD0000FFFF000078
:10B1B00038B50024E44389B280B26B46042200F023
:10B1C00011F8002806D103216846435C2202D418F6
:10B1D000491EFAD5204638BD10B500210846FFF7B4
:10B1E000E7FF10BD38B5002909D0402420436C4644
:10B1F0002070C8B27F2906D8607002200AE0694634
:10B200000870012006E0802420436C466070C80965
:10B21000A0700320694600F0B1FF38BD10B5144698
:10B2200003460A4621461120FFF7DCFF10BD10B58A
:10B230000346052200211520FFF7D4FF10BD10B5ED
:10B240000346052200211720FFF7CCFF10BD38B5BB
:10B25000054600206946087000F0C4F8FF24013458
:10B260002246002D01D00322120200210D2000F001
:10B27000D3F8002D13D06B46012203210F20FFF7D6
:10B28000B1FF68460078000709D5FFF7A3FE224604
:10B2900000210D2000F0C0F80020C04338BD002080
:10B2A00038BD10B5024601210A2000F0C0F810BDDB
:10B2B00010B5044600211A20FFF77AFF000D220383
:10B2C0000005120B024300211A2000F0B0F810BD57
:10B2D00010B5024602492E2000F09EF810BD000075
:10B2E00004180000F8B505466B460122032104202E
:10B2F000FFF778FF0126114C3607002D0DD02A46A6
:10B3000000210C2000F088F86946087810210843D5
:10B3100069460870A069304307E069460878EF2164
:10B32000084069460870A069B0430B46A06101223D
:10B330000321042000F08AF8F8BD0000BC010020C1
:10B3400010B502460021182000F066F810BD00007C
:10B35000F8B50746002568460570B807204C2E460C
:10B3600000280ADA8020694608706B460122002115
:10B370000D2000F06BF801202073F807694608786B
:10B3800021D006210843694608706B46012200213E
:10B390000D2000F05BF803210F20FFF7F3FE812161
:10B3A000C900084219D04020694608706B46012246
:10B3B00000210D2000F04AF80020FFF7F7FD0025DE
:10B3C0002673ED4309E002210843694608706B4685
:10B3D000012200210D2000F039F82846F8BD0000B8
:10B3E000DC0100201CB56B46012203210F20FFF772
:10B3F000F9FE684600784022C1091040C9014000AA
:10B40000814208D0012069460871024601AB032140
:10B410000D2000F01BF81CBD08B56B461A70120A0F
:10B420005A7089B280B2022200F010F808BD38B517
:10B4300000236C46E254120A5B1C042BFADB89B22F
:10B4400080B22346042200F001F838BD38B58024CC
:10B45000002909D0C02528436D462870C8B27F292D
:10B4600007D86870022009E020436946087001206F
:10B4700004E020436870C809A8700320694600F002
:10B4800027FF38BD10B51446012312189B029A42BB
:10B4900002D90020C04310BD0B46821E2146092060
:10B4A000FFF7D4FF002010BD10B5054A89051269C9
:10B4B00001430A4300210820FFF7B9FF002010BD17
:10B4C000BC01002038B504466B4601220E212B201A
:10B4D000FFF788FE68460078E10640094001C90E82
:10B4E0000143684601706B4601220E212B20FFF7B5
:10B4F000ADFF38BD10B5002142541C06120A22438C
:10B500001B0A491C0429F7DB10BD000013B50123F9
:10B510001A4669460248FCF765FD00981CBD00000C
:10B52000CC1600207CB5002425466846FFF77FFE38
:10B5300004206946220E2D02154322020C5C14439E
:10B54000401EF7D5204629467CBD7CB50024254603
:10B550006846FFF774FE04206946220E2D0215434B
:10B5600022020C5C1443401EF7D5204629467CBDC0
:10B57000FBF78AFBFEF7C4F9FDF70AF93E493F489D
:10B58000002522C005608561C5613D490562C16035
:10B590000838FBF70BFDFDF7E7F8FDF7BFF9FDF7FE
:10B5A0009BF9FDF7ADF8052401222407D1032046BD
:10B5B000FBF755FBFDF750FFFCF78AFFFAF746FB58
:10B5C000FAF7C8FBFAF796FBFCF78EFD0721A015EA
:10B5D000FFF7D4FCFFF7E6FC012211032046FBF73E
:10B5E0003EFB2648C8222749C830FCF7C9FC264F35
:10B5F000264E274C387800280FD13078002801D00B
:10B6000003280AD10121C9022248FBF71BFB0028AD
:10B6100003D101210846FBF7DDFDE078002828D0A2
:10B620006078002825D0E57072B620780F280AD9F6
:10B630000120184900038861FEF7E6F90120154949
:10B64000000388620CE0012251031248FBF707FB5C
:10B65000FEF7DAF90121002249030E48FBF7FFFA51
:10B6600062B6FCF75FFE208C0028C3D0401E208409
:10B67000C0E7FCF757FEBDE7007C00400416002041
:10B68000FFFF0000200D00205A0000208400002051
:10B690003C0100200004005010B586B01748FBF7AD
:10B6A00008FC14216846F9F782FD15480090032034
:10B6B000019000200290052069460007FBF706FA7A
:10B6C00069461048FBF702FA69460F48FBF7FEF996
:10B6D00001210846FBF77EFDFF2401342046FBF7DD
:10B6E00051FD0A4908680422104308602046FBF710
:10B6F00059FDFBF75FFD06B010BD000004160020E9
:10B70000FFFF0000000400500008005000700040DF
:10B7100010B50122920217491748FAF79FFB154806
:10B72000164902888A4223D0018004218180FF21AA
:10B73000F531C1800A21018100211E224181D243BD
:10B7400082810122C28181834323C386022303872E
:10B75000782343878287C28702464032118451840E
:10B760009184C183918014238382118200F02CFD87
:10B7700010BD0000E80D002000FC0008AA550000E4
:10B78000F0B51FB496B084460C460246199D189831
:10B790000390490068006300490840080193002AAB
:10B7A00001D0012600E000269E19FE4BF6185B1022
:10B7B0009E422BD36E00039F0296002F00D00127DC
:10B7C000F719F84EF84BBE199E421FD3039E03464D
:10B7D000F64F334309D03B469C4201D1002A04D0A6
:10B7E000019B002A05D0012604E0002039461BB049
:10B7F000F0BD00269E19EE4B9E4207D8039F029E85
:10B80000002F00D00127F6199E4207D92B4660462B
:10B810002146189AFEF788FE1BB0F0BD0023002CCD
:10B8200029DAE44EB04226DAE34EB04201DB0223CD
:10B8300021E0DE4EB0421EDBE04E070DBE19142E95
:10B8400009DD3427BF1B039EFE400196BE40039FC7
:10B85000BE420BD00FE0039F002F0CD11427BF1B5B
:10B860000646FE400196BE40864204D1019BDE079B
:10B87000F60F02239B1B0E46164318D1002D16DA35
:10B88000002C03D0022B01D0012B06D00220FEF7A2
:10B890007BFEFEF73FFE1BB0F0BD0220FEF774FEFC
:10B8A000FEF738FE0122D20751401BB0F0BD039EC7
:10B8B000002E61D1BF4EB04220D1C148844201D197
:10B8C000002A08D0B948814209DB002D10DB189806
:10B8D00029461BB0F0BD0020B4491BB0F0BD002DBF
:10B8E00006DA01222946D207189851401BB0F0BD54
:10B8F000B4497944086849681BB0F0BDAB4FB84201
:10B9000025D1002D1FDA002904D0B14212D1002A1E
:10B9100009D018E0002A72D1A649E20F0020D20710
:10B9200011431BB0F0BD0020E20F0146D2071143C6
:10B930001BB0F0BDB14206DA234600203946F9F7C4
:10B9400049FE1BB0F0BD104621461BB0F0BDB14210
:10B9500012DA0126B607B54203D12346104619462E
:10B96000FEE3994EB54207D1261E05DB104631464F
:10B9700000F040FC1BB0F0BD67007F081646002AAF
:10B9800040D100290AD08B4A914229D1002C0EDDEA
:10B99000002D1CDB002011461BB0F0BD022B16D081
:10B9A000002C14D0012B12D1002C14DB0FE0002C42
:10B9B00028DA002D09DB012B03D000207D491BB0C4
:10B9C000F0BD002081491BB0F0BD012B03D0002049
:10B9D00001461BB0F0BD00200121C9071BB0F0BD1E
:10B9E000724A91420ED1002C01DA002B17D0022BA3
:10B9F00006D00020C043F9F78DFE1BB0F0BD90E2E9
:10BA00000120F8E7E217521C94461A4307D000229F
:10BA10000892664C62465B1E1A4307D009E001207B
:10BA2000FEF7B2FDFEF784FD1BB0F0BD0022644CB2
:10BA30000892674A90427DDD664B674A98421FDD57
:10BA4000914202DC002D05DB4DE05848814217DBB6
:10BA5000002D48DD0220FEF797FDFEF771FD05463B
:10BA60000E460022534B21460898F9F74BFD084635
:10BA700071004908C00FC007014328461BB0F0BD44
:10BA8000914215DA002D2EDA0220FEF77DFDFEF739
:10BA900057FD05460E460022464B21460898F9F709
:10BAA00031FD72005208C80FC0070243114617E06B
:10BAB0003E4B994223DD002D15DD0220FEF764FD8B
:10BAC000FEF73EFD05460E4600223A4B21460898F9
:10BAD000F9F718FD084671004908C00FC007014377
:10BAE00028461BB0F0BD0220FEF74EFDFEF732FDEA
:10BAF00049004908E20FD20711431BB0F0BD0022F4
:10BB000030463946F9F7F0FC012205460E46D2438D
:10BB1000F9F7D8FD314A324BF9F7ECFC2A463346A7
:10BB2000F9F7F0FC0022284BF9F7E4FC07462A4617
:10BB3000334600E064E0039110461946F9F7E2FC51
:10BB40003A46039BF9F7DEFC0746032209915207A8
:10BB5000244B28463146F9F7D5FC07910C90224A30
:10BB6000204B38460999F9F7CDFC074601911F4A49
:10BB70001F4B28463146F9F7C5FC3A46019BF9F7B9
:10BB8000B3FC07460B460246099107990C98F9F752
:10BB900007FC00250E462846079B0C9AF9F7A4FCE3
:10BBA0003A4627E0FFFF1F00FFFF0F000000F03FB5
:10BBB0000000E0FF0000F07F0000404301FCFFFFB9
:10BBC0000000F0BF5A0B00000000E03F0000F0FF53
:10BBD0000000E0410000F043FFFFEF3F5555555591
:10BBE0005555D53F4715F73FFE822B6544DF5DF87D
:10BBF0000BAE543E099BF9F77DFC02460B4652E121
:10BC0000012500202D05A94207DA352230463946A4
:10BC1000F9F758FD06463420C0430A151218FE48AD
:10BC2000101803900803FD49000B01430F46FC491F
:10BC3000884201DC002003E0FA49884202DA012050
:10BC4000119005E0002011900398401C7F1B039089
:10BC500011980597C200F4480F9278448018436801
:10BC60000268394630460D930292F9F73DFC079180
:10BC70000C9030460D9B029A0599F9F791FB02460C
:10BC80000B460020E549F9F7A5FC09910490079BB4
:10BC90000C9AF9F737FC129000201090E3480D46FB
:10BCA000784400680E9001217810490708431199E3
:10BCB0000D9B890440180121C90447183946029A8E
:10BCC0000E98F9F711FC3246059BF9F713FC024672
:10BCD0000B4629461098F9F715FC064602913B469B
:10BCE00029460E9A1098F9F70DFC079B0C9AF9F764
:10BCF00001FC3246029BF9F7F7FB099B049AF9F71E
:10BD000001FC0591129A0A902B4610461946F9F744
:10BD1000F9FB06460246C6480F460B460621784404
:10BD2000FEF7A2FB32463B460091049010461946AE
:10BD3000F9F7E8FB009B049AF9F7E4FB06460F4687
:10BD40002B461946129A1098F9F72AFB059B0A9A76
:10BD5000F9F7D8FB32463B46F9F722FB109A0791D8
:10BD600004902B4610461946F9F7CCFBB14E002241
:10BD7000334609910290F9F713FB079B049AF9F7F0
:10BD80000FFB00200746024633460091F9F7ACFB53
:10BD9000099B029AF9F7A8FB079B049AF9F7AAFBFB
:10BDA00006460D913A462946009B1098F9F7AAFBE2
:10BDB00007910C902B463046129A0D99F9F7A2FB89
:10BDC00005460E463A46009B05990A98F9F79AFBF4
:10BDD00033462A46F9F7E4FA02460B46074609912C
:10BDE00007990C98F9F7DCFA00250E462846079BC0
:10BDF0000C9AF9F779FB3A46099BF9F77BFB074662
:10BE00000722099152078C4B31462846F9F77AFBF5
:10BE100007910090894A884B38460999F9F772FBD7
:10BE200007460191864A874B31462846F9F76AFB57
:10BE30003A46019BF9F7B4FA834B7B440F9A9B185F
:10BE40001A685B68F9F7ACFA029009910398F9F760
:10BE500061FC05910490099B029A07990098F9F7F3
:10BE60009FFA7A4B7B440F9A9B181A685B681746B7
:10BE70000393F9F795FA059B049AF9F791FA0E46A0
:10BE80002846059B049AF9F72FFB3A46039BF9F7DE
:10BE90002BFB079B009AF9F727FB099B029AF9F7FE
:10BEA00029FB02460B46199900200C900F46189862
:10BEB000F9F728FB029104903B460C9A19991898BF
:10BEC000F9F712FB2A463346F9F71CFB029B049A4A
:10BED000F9F766FA09910E902A46334639460C98CE
:10BEE000F9F710FB06460F46099B0E9AF9F758FA28
:10BEF000574A0D46914220DB5242AA18024310D104
:10BF000032463B46F9F7F0FA04900391514A524BFE
:10BF100009990E98F9F744FA039B049AF9F7B4FCCF
:10BF20001ED20220FEF730FBFEF70AFB490049084B
:10BF3000E20FD20711431BB0F0BD6A00474B520815
:10BF40009A420DD3464AAA18024300D0CBE53246A6
:10BF50003B46F9F7C9FA099B0E9AF9F795FCF5D912
:10BF60006800002340082C490393020D3D4B5218F2
:10BF7000984223DD01200005521CD0404219500098
:10BF8000400D401838497944096813468C463749B2
:10BF9000C1408B4312030121120B090551181422D1
:10BFA000101AC1400391002D01DA48420390624605
:10BFB00030463946F9F798FA06460F4632463B4670
:10BFC00009990E98F9F7ECF900252A46284B2846DE
:10BFD0000591F9F797FA07910C90264A264B2846C7
:10BFE0000599F9F78FFA0091029032463B462846B0
:10BFF0000599F9F779FA099B0E9AF9F77BFA1F4A26
:10C000001F4BF9F77FFA009B029AF9F7C9F9074627
:10C010000B460246099135E001FCFFFF0000F03FAE
:10C020008E9803007AB60B006A070000AC07000088
:10C03000D60600000000084009C7EE3FFD033ADCC9
:10C04000F5015B14E02F3EBEAA050000700500005C
:10C0500000009040FE822B654715973C00CC904035
:10C0600000346F3F0000E03FC6040000FFFF0F00F8
:10C07000432EE63F396CA80C615C20BEEF39FAFE16
:10C08000422EE63F07990C98F9F78AF905460E46C5
:10C09000079B0C9AF9F728FA3A46099BF9F72AFA0E
:10C0A00009912A4633460E9010461946F9F72AFAA6
:10C0B000074602462F480B46059105217844FEF7B6
:10C0C000D3F93A46059BF9F71DFA2A463346F9F7A4
:10C0D00011FA0746019128463146099B0E9AF9F755
:10C0E00011FA099B0E9AF9F75BF9012304910C9060
:10C0F00000229B0738460199F9F7F6F905910E9051
:10C100003A4628463146019BF9F7FCF9059B0E9A01
:10C11000F9F760FA049B0C9AF9F7E6F92A463346D8
:10C12000F9F7E2F90022144BF9F7E4F9064603980F
:10C130000D46000541190915002912DC3046294633
:10C14000039AF9F7BFFAFEF749F9042801D1FEF77F
:10C1500001FA30462946039AF9F7B4FA064601E097
:10C1600004E029180B46324621460898F9F7CAF927
:10C170001BB0F0BD680300000000F03FF0B58C4636
:10C1800000251026052109078E620E4C08E067463F
:10C190007F5DE760A768FF07FCD0E7681F706D1C34
:10C1A0008542F4DB0020074606E0E760A568ED075E
:10C1B000FCD0E5681D54401C9042F6D38E610020EF
:10C1C000F0BD00000030014070B572B60124074D8B
:10C1D000A40221462846F9F727FE002804D022466B
:10C1E00003492846F9F7C4FE62B670BD00FC00089A
:10C1F000E80D0020F8B506460C46F9F753FC051E7D
:10C200000F4600D00120014349000B484908411A5C
:10C21000C90F0DD0002E01D0012100E000210C43F8
:10C2200061004908401AC00F02D10120FEF7ACF9A5
:10C2300028463946F8BD00000000F07FF8B51546E5
:10C240000E460746002407E03819C0B200F008F88F
:10C25000641C2870E4B26D1CB442F5D33046F8BDBE
:10C2600010B50446FBF7FAFFEE20FBF7CAFFFCF718
:10C270002EF82046FBF7C5FFFCF729F8FBF7EEFF89
:10C28000EF20FBF7BEFFFCF722F80020FBF78CFF46
:10C290000446FBF7FEFF204610BD704770B50D4603
:10C2A0000446FBF7DBFFEE20FBF7ABFFFCF70FF8D4
:10C2B0002046FBF7A6FFFCF70AF82846FBF7A1FF8C
:10C2C000FCF705F8FBF7E5FF0A20FEF7A6FA70BDBC
:10C2D000F0B50025102605279C463F070B46BE6299
:10C2E0000C4C06E0595DE160A168C907FCD0E1682B
:10C2F0006D1C8542F6DB002007E06146095CE160C9
:10C30000A168C907FCD0E168401C9042F5D3BE612A
:10C310000020F0BD003001400000010203040005D0
:10C32000405C0000A05C0400C06C0800805C04005D
:10C33000E03F1E00E07D1E0007A9022570889B8853
:10C340000A001600010006000100020087008D00AF
:10C350002D001A3152001A339A001A351D011A376E
:10C360006B003B31BE003B335E013B3596023B37F1
:10C37000000099599959EB518F421E45142E0080A7
:10C38000EB51F5283333E13A703DE13AC235852B64
:10C39000C2353333C235C235AE47E13A5138A330E6
:10C3A00051380000000000000000010203040607ED
:10C3B0000809030406080C101820300000000001D2
:10C3C0000203040000000000000000000000F03F35
:10C3D000000000000000F83F000000000000000026
:10C3E0000000004003B8E23F000000000000000031
:10C3F00006D0CF43EBFD4C3E033333333333E33FBF
:10C40000FFAB6FDBB66DDB3F4D268F515555D53FEA
:10C4100001411DA96074D13F65DBC9934A86CD3FB8
:10C42000EF4E454A287ECA3F3E5555555555C53FA6
:10C4300093BDBE166CC166BF2CDE25AF6A56113F98
:10C44000F16BD2C541BDBBBED0A4BE726937663E9A
:10C45000000000000000000078C400080000002078
:10C46000900100006C5B0008DCC400089001002013
:10C47000681A000078A500080124130704380D0984
:10C480001E080540082609104008560A131D043BE3
:10C4900008BE0516D8BC4010085201033AC842072E
:10C4A0007052030CE5800C1B0202DD14090102220C
:10C4B00081F01F6681049889968696798215980383
:10C4C000981498879674977882439788967197778F
:0CC4D0008249F10139293F9204922000BA
:04000005080050C1DE
:00000001FF
